:100000000C94D5050C94F2050C94F2050C94F205B1
:100010000C94F2050C94F2050C94F2050C94F20584
:100020000C94F2050C94F2050C94F2050C94F20574
:100030000C9459070C94F2050C94F2050C94DC070F
:100040000C949C060C94F2050C948B530C94F205C2
:100050000C94F2050C94F2050C94F2050C94F20544
:100060000C94F2050C94BB060C94F2050C94F2056A
:100070000C94F2050C94F2050C94F2050C94F20524
:100080000C94F2050C94F2050C94F20552554420A0
:10009000454C45205448522041494C20525544205B
:1000A00054485220454C452041494C2041494C2060
:1000B000454C4520544852205255442041494C203B
:1000C00054485220454C452052554420000301021B
:1000D00000040506070000000000011E6401011E67
:1000E00064010132960A0A32966D656E7553746129
:1000F000636B206F766572666C6F77006D656E75E9
:10010000537461636B20756E646572666C6F770003
:100110005B4D454E555D20205B455849545D0020A0
:100120005945532020202020204E4F20200070725F
:1001300065737320616E79204B657900414C45529F
:100140005400544852206E6F742069646C650045F9
:100150004550524F4D206C6F77206D656D004F46B6
:1001600046414253525573525525454C73454C25D3
:10017000544873544825414C73414C25503120500C
:100180003125503220503225503320503325005431
:100190004852525544454C454944304944314944FC
:1001A0003241494C47454154524E535731535732CF
:1001B000535733535734535735535736004F4646EA
:1001C000004F4E20002D2D2D002D2D2D2043483188
:1001D00020434832204348332043483420434835A5
:1001E0002043483620434837204348382043483985
:1001F000204348313043483131434831324348315C
:10020000334348313443483135434831364348312C
:100210003743483138434831394348323043483214
:100220003143483232434832334348323443483210
:1002300035434832364348323743483238434832F0
:100240003943483330005031202050322020503381
:1002500020204D41582046554C4C50504D31505067
:100260004D3250504D3350504D3450504D3550500C
:100270004D3650504D3750504D384348312043484B
:1002800032204348332043483420434835204348F4
:1002900036204348372043483820434839204348D4
:1002A0003130434831314348313243483133434898
:1002B0003134434831354348313643483137434878
:1002C000313843483139434832304348323143486A
:1002D000323243483233434832344348323543485C
:1002E000323643483237434832384348323943483C
:1002F0003330002D2D2D2D00564552533A205631C6
:100300002E323937392D6B747300444154453A20ED
:1003100030312E31302E323031300054494D453A93
:100320002031303A31303A3332002053564E3A20A1
:100330007472756E6B2D7231383900120812000814
:100340001C0808081C0800000822004900220800B8
:1003500000000000227F2200000008220049002245
:1003600008000008220049002208000000227F2225
:100370000000000000082200490022080000081CBC
:100380000808081C08004637D727152C8C3B662F19
:10039000963D452EBD42CC3119345927CC34FD341D
:1003A0009F35113670756C736520746162206F76AD
:1003B0006572666C6F7700544852525544454C45FF
:1003C00049443049443149443241494C47454154FC
:1003D000524E535731535732535733535734535761
:1003E0003553573600544852525544454C454944BC
:1003F0003049443149443241494C47454154524EB9
:100400005357315357325357335357345357355348
:1004100057360020202054546D00457870457846AA
:10042000466E654D656443727300544F54005354D7
:10043000250053544B0054535700544D450053541A
:100440004154004A45544900746D61696E20202072
:10045000202020202020206D7300746D7231204AEE
:10046000697474657220202020757300746D723178
:100470004C6174206D696E20202020757300746DAE
:1004800072314C6174206D617820202020757300DA
:100490005354415432004D6F64650020524554411D
:1004A00000205245544100205245544100205245FD
:1004B0005441004368616E6E656C204F72646572D2
:1004C000004F4646007320004C69676874204F4611
:1004D00046206166746572004C69676874205357E2
:1004E000004F4646204F4E005468726F74746C651E
:1004F000205265760053494E474F534D5046494C64
:10050000540046696C74657220414443006D204973
:100510006E616374697669747920416C726D0056FE
:1005200020424154205761726E696E6700436F6EBE
:100530007472617374005345545550004F46460021
:100540004F4E00544852205761726E535720205727
:1005500061726E4D454D205761726E4265657065E2
:10056000722020005345545550204F50545300439F
:10057000616C0050504D494E00010456455253499C
:100580004F4E005472696D2D202B00204D656E7505
:10059000204578697420446F776E20202055705272
:1005A00069676874204C656674004449414700419E
:1005B00031413241334134413541364137413800D0
:1005C000414E41003C202020203E005365744D697F
:1005D00064205365745370616E446F6E65202020F3
:1005E0000043414C494200312F3800667265650076
:1005F0004D4F44454C53454C0044454C45544520D3
:100600004D4F44454C2020205B4D454E555D0050DC
:100610004F534E45470053686966742053656C001C
:1006200075536563003443482036434820384348B7
:100630002031304348313243483134434831364326
:10064000480050504D20202053494C565F4153499B
:100650004C565F4253494C565F43545241433039E4
:100660000050726F746F0052455441313233004272
:1006700065657020436E74005472696D2053770075
:10068000457870202020457846696E6546696E651C
:1006900020204D656469756D436F61727365005408
:1006A00072696D20496E63004F46464F4E200054DC
:1006B0002D4578706F004F46464F4E2000542D5404
:1006C00072696D00436F756E7420446F776E436F6F
:1006D000756E7420557020200054696D657220007D
:1006E000547269676765720054696D6572004E6186
:1006F0006D650053455455502000010A0201010167
:100700000101010703010120414243444546474896
:10071000494A4B4C4D4E4F505152535455565758D1
:10072000595A303132333435363738395F2D2E004F
:100730006578702020252020737731207377320070
:100740004558504F2F4452000504445220486967D1
:1007500068004452204C6F77004452204D69640079
:10076000447253773200447253773100576569679A
:100770006874004578706F004558504F2F445220E0
:10078000002D2D2D783E30783C307C787C663E30D4
:10079000663C307C667C63312063322063332063A7
:1007A0003420633520633620633720633820633973
:1007B000206331306331316331326331336331343B
:1007C000633135633136002B2A52007774207372FF
:1007D000632020737720637276004D49584552009C
:1007E00044454C455445204D4958205B4D454E5598
:1007F0005D00536C6F772020557000536C6F77202D
:1008000020446F776E0044656C6179205570004418
:10081000656C617920446F776E004164642020200C
:1008200020204D756C7469706C795265706C6163D1
:100830006520004D756C747078004F464600576116
:10084000726E696E6700537769746368002D2D2D91
:10085000783E30783C307C787C663E30663C307C3C
:10086000667C633120633220633320633420633538
:1008700020633620633720633820633920633130AA
:100880006331316331326331336331346331356322
:10089000313600437572766573004F4E204F4646E1
:1008A000005472696D004F66667365740057656920
:1008B00067687400536F757263650045444954203E
:1008C0004D49582000494E53455254204D49582017
:1008D000002D2D2D2D202020763E6F667320207652
:1008E0003C6F667320207C767C3E6F66737C767CE2
:1008F0003C6F66730073726320206F6673206675A9
:100900006E630043535749544348000303434C4527
:100910004152204D49584553205B4D454E555D0091
:1009200054454D504C4154455300434F5059205469
:1009300052494D205B4D454E555D002D2D2D494EA4
:10094000560073756254206D696E20206D617820A9
:10095000696E76004C494D495453000104435600DA
:100960004355525645005052455345540043555245
:1009700056452000454550524F4D206F76657266B2
:100980006C6F7700454550524F4D206F766572660B
:100990006C6F770067656E77726974652065727237
:1009A0006F720042616420454570726F6D20446132
:1009B0007461004D4F44454C2020202020005008F9
:1009C00050000000000000005E000000080608065D
:1009D000287E287E28042A7E2A104C2C1068643435
:1009E0004A5620500000000806000018244200006B
:1009F00042241814083E081408083E08080000B0F5
:100A00007000000808080800006060000060180618
:100A100000003C42423C0000447E40004462524C94
:100A200000424A4A340018147A10002E4A4A320012
:100A30003C4A4A300002720A0600344A4A34000C2A
:100A400052523C00006C6C000000A86800000008D6
:100A50001422001414141400002214080004520A72
:100A6000043C425A5A1C007C12127C007E4A4A34D2
:100A7000003C424224007E42423C007E4A4A420000
:100A80007E0A0A02003C425234007E10107E004270
:100A90007E4200002040403E007E182442007E40FE
:100AA00040407E0408047E007E08107E003C4242E6
:100AB0003C007E12120C003C42225C007E12324C42
:100AC00000244A522402027E0202003E40403E1EA2
:100AD0002040201E7E2018207E422418244202043A
:100AE0007804020062524A46007E42420000061824
:100AF00060000042427E000804020408404040407A
:100B00004000000608000030484878007E48483021
:100B10000030484848003048487E0078485858001F
:100B200008FE0A080010A8A878007E08087000488F
:100B30007A4000008088FA00007E10284000427E43
:100B40004000780870087000780808700030484845
:100B50003000F828281000102828F800781008081D
:100B6000005058682800087E4848003840407818EF
:100B70002040201838403040380048303048009835
:100B8000A0A078004868584800107C440000007E0F
:100B900000000000447C101010443810103844103D
:100BA0001040800804201002010011241FBECFEF66
:100BB000D0E1DEBFCDBF12E0A0E0B1E0ECEAF9EA9F
:100BC00002C005900D92AA37B107D9F710E1AAE744
:100BD000B2E001C01D92A630B107E1F70E94F80C07
:100BE0000C94D4540C940000E0913C05F0E0EE0F1E
:100BF000FF1FEC5CFA4F808191810895FC01A09168
:100C00003C05B0E0AA0FBB1FAE5CBA4FED93FC935E
:100C10008FEB099580913E0580933D050895E82F5F
:100C2000F0E0E353FF4FE491F0E0EE0FFF1FED57CC
:100C3000FA4F8FB7F8942081318187FF01C07894F3
:100C4000C9010895A3E8B5E0E3E9F5E020E0822FCB
:100C5000806487B9369A349BFECF349A6089718953
:100C60008D919C91119796958795860F971F8E7FF2
:100C70008D939D9340815181CB01840F951F969553
:100C80008795918B808B84B195B1840F951F969534
:100C90008795819391932F5F2830C9F60895DF934C
:100CA000CF93CDB7DEB760970FB6F894DEBF0FBE17
:100CB000CDBFFE01319680E1DF011D928A95E9F7F3
:100CC000A3E8B5E080E015C047B9369A349BFECF63
:100CD000349A64B175B1260F371F9F5F9430A1F726
:100CE00021933193369527952D933D938F5F8830CF
:100CF00031F02081318190E0482F4064E5CF60964B
:100D00000FB6F894DEBF0FBECDBFCF91DF9108952F
:100D1000E3E8F5E080E0982F906497B9369A349B29
:100D2000FECF349A24B135B1220F331F2193319372
:100D30008F5F883081F708951F920F920FB60F9240
:100D400011248F9380917F058F5F80937F058F9112
:100D50000F900FBE0F901F90189530917F0522B70E
:100D600080917F053817C9F7932F80E030E0282B5A
:100D7000392BC901089578941F920F920FB60F92E4
:100D800011242F933F934F935F936F937F938F9390
:100D90009F93EF93FF932091800030918100F8940E
:100DA00080917D008F7D80937D00789480916B058C
:100DB0008F5F8F7090916C05891789F4E0916B05B6
:100DC000F0E03F96EF70F070EE0FFF1FE55BFA4F1B
:100DD000118210828091410580933D0513C0E091FE
:100DE0006B05F0E04091800550918105B901641BCD
:100DF000750BAB01EE0FFF1FE55BFA4F518340838C
:100E000080936B053093810520938005F894809141
:100E10007D00806280937D007894FF91EF919F9197
:100E20008F917F916F915F914F913F912F910F9093
:100E30000FBE0F901F90189580917D0531C0E091F5
:100E40006C05F0E0EE0FFF1FE55BFA4F208131816A
:100E50003695279590916C059F5F9F7090936C05D8
:100E6000982F91509830A8F4A9014152534095E031
:100E70004737590710F080E013C0E82FF0E0EE0F7D
:100E8000FF1FE559FA4F2C5D3540318320838F5F7A
:100E900007C0215A3F409EE22F3D390708F481E008
:100EA00020916C0590916B05291749F680937D057B
:100EB00008951F920F920FB60F9211242F933F9314
:100EC0004F935F936F937F938F939F93AF93BF9352
:100ED000EF93FF9380E09CB59A3008F065C08F5F78
:100EE0008233C9F761C0C09A1092C30504C0C0988C
:100EF00021E02093C3055091CA074091CB07252FCD
:100F0000342F2817390708F49C013093CB0720931E
:100F1000CA075091080140910901252F342F8217EB
:100F2000930708F49C013093090120930801A091D4
:100F30000601B0910701FD01819191919BBD8ABD90
:100F4000F0930701E093060112968D919C911397FF
:100F50000097A1F48EEC97E090930701809306012F
:100F60008091DC028093C30587B78F7E87BF78941A
:100F70000E944812F89487B7806187BF80917E05F0
:100F8000816080937E05FF91EF91BF91AF919F911A
:100F90008F917F916F915F914F913F912F910F9022
:100FA0000FBE0F901F9018958CB59DB52091C3056D
:100FB000222309F098CF9BCF78941F920F920FB6FF
:100FC0000F9211242F933F934F935F936F937F93CF
:100FD0008F939F93AF93BF93EF93FF93F89487B74B
:100FE0008D7F87BF789481B7845681BF80913D05FE
:100FF000882399F0815080933D05809131058823A5
:1010000021F08091820591E08927809382058823D1
:1010100011F01B9805C01B9A03C01B981092310554
:101020000E94194E80917E05826080937E05F8941F
:1010300087B7826087BF7894FF91EF91BF91AF919E
:101040009F918F917F916F915F914F913F912F91E0
:101050000F900FBE0F901F901895803F09F4BDC0F0
:10106000882309F4BBC0803109F4B5C0282F332789
:1010700027FD3095B90137FF04C066277727621B2B
:10108000730B6A308CF418164CF08DE090E0821BE4
:10109000930B0E947B4D61E06827A0C0C9010D96AB
:1010A0000E947B4D682F9AC0772767FD70956A5024
:1010B0007040FB01EE0FFF1FE60FF71FE45EFA4FD3
:1010C0009081915009F489C0983038F4E92FF0E00C
:1010D000EE0FFF1FE753FA4F1EC09A3018F420E0BE
:1010E00034E01BC0E92FF0E0913188F4DF01AA0F52
:1010F000BB1FA55ABA4FEE0FFF1FE656FD4F2D91AD
:101100003C91119740815181241B350B06C0EE0F95
:10111000FF1FEB54FA4F20813181FB01EE0FFF1FBF
:10112000E60FF71FE35EFA4F9081492F97FD4D5F61
:1011300045954595552747FD5095EAE09E02F001FB
:1011400011244E0F5F1FFB01EE0FFF1FE60FF71F6D
:10115000E25EFA4F9081913039F0923059F093303D
:1011600079F09430D1F522C0181614F460E010C064
:1011700060E018C0181614F460E020C060E028C0D9
:10118000181654F460E037FF03C0309521953F4FA7
:10119000421753071CF51FC060E037FF03C03095AE
:1011A00021953F4F42175307CCF015C0181654F441
:1011B00060E037FF03C0309521953F4F2417350776
:1011C0006CF409C060E037FF03C0309521953F4FB4
:1011D000241735071CF061E001C060E0862F0895F8
:1011E0002F923F924F925F927F928F929F92AF92F7
:1011F000BF92CF92DF92EF92FF920F931F93DF93F4
:10120000CF930F92CDB7DEB7182F1B017A0169017A
:10121000702E802F90E064E0462E512C48225922F7
:1012200002FF04C0F101A080B18005C0F101A080DF
:10123000BB24A7FCB09483FD03C025E004E002C0FA
:1012400022E003E014FF05C01F701066802F022FFC
:10125000282F802F8066181761F0802F8064181760
:1012600041F08091F805882371F0133611F01334A2
:1012700051F445010894811C911C80913E05809396
:101280003D05822F19C0922F9066191761F0922F99
:101290009064191741F0882309F46FC0123619F0D1
:1012A000123409F06AC045010894810891088091C0
:1012B0003E0580933D05802F90E029830E947B4D61
:1012C0002981882351F0882499248A189B08822F29
:1012D0000E94F74D802F0E94F74D80914505909117
:1012E0004605881A990AC814D90444F4812F0E942B
:1012F000F74D8091400580933D0546018E149F0473
:1013000044F4812F0E94F74D8091400580933D0564
:1013100047018A149B04D9F08114910439F4812F78
:101320000E94E84D80913E0580933D054114510493
:1013300021F0F1019182808202C0F1018082872D2B
:1013400083700E94624381E08093420503C0109243
:10135000420580E00F90CF91DF911F910F91FF9098
:10136000EF90DF90CF90BF90AF909F908F907F9045
:101370005F904F903F902F9008954501AECF0F930F
:10138000DF93CF930F92CDB7DEB76983552747FD23
:101390005095332727FD3095BE016F5F7F4F09E0E1
:1013A0000E94F00889810F90CF91DF910F910895ED
:1013B0000F93DF93CF930F92CDB7DEB76983552795
:1013C00047FD5095332727FD3095BE016F5F7F4F56
:1013D00001E00E94F00889810F90CF91DF910F9179
:1013E00008950F93DF93CF930F92CDB7DEB7698344
:1013F000552747FD5095332727FD3095BE016F5F78
:101400007F4F0AE00E94F00889810F90CF91DF9111
:101410000F9108950F93DF93CF930F92CDB7DEB75F
:101420006983552747FD5095332727FD3095BE0129
:101430006F5F7F4F02E00E94F00889810F90CF918B
:10144000DF910F9108951F93182F8F708650909100
:10145000D802923074F0492F552747FD50954150DE
:10146000504021E030E002C0220F331F4A95E2F7DE
:10147000922F883008F08FC016FF8DC0282F259539
:10148000992399F4E22FF0E0E855FB4F408155276E
:1014900047FD509557FF03C0509541955F4F942FDE
:1014A00047FD9D5F959595959F5F30E06091BE02E9
:1014B00070E06170707042E050E0461B570B4217BD
:1014C000530739F44091D7024F7019F051E094E07E
:1014D00001C050E0692F772767FD7095F901EA5345
:1014E000FD4F80FF09C0EE51FE4F8081992787FD97
:1014F0009095860F971F08C0EE51FE4F8081992767
:1015000087FD9095861B970B009771F0492F4095AA
:10151000441F4427441F60E0F901E855FB4F7081E8
:1015200077FF61E0461769F0552359F4F901E85552
:10153000FB4F4081442329F01082812F0E94F74DF8
:1015400023C0AC0144585F4F493F510580F42855F2
:101550003B4FF901808382E00E94624316541830A9
:1015600018F481E08093310580913F0511C0181671
:10157000190614F083E801C08DE728553B4FF901A7
:10158000808382E00E946243109231058091400581
:1015900080933D0510E0812F1F9108954091E00F49
:1015A0005091E10F80E02091C7053091C8054217A6
:1015B000530709F081E0809348058091E00F9091F6
:1015C000E10F9093C8058093C7058AEF95E060E02E
:1015D00040E00E945D1480E00E9472430E94D14C62
:1015E0000E94FB4C0E94230A482F809148058823C3
:1015F00059F08091490590914A05009729F001978B
:1016000090934A0580934905842F807F803289F426
:101610008091C20290E024EF31E0BC01629FC001E2
:10162000639F900D729F900D112490934A058093B3
:1016300049052091D5053091D605809143059091BB
:101640004405821B930B60E270E00E944254709349
:101650004605609345056115710591F08091C505BA
:101660009091C605821B930B62E070E00E94425489
:1016700070934605609345053093440520934305D8
:101680003093C6052093C505E0913C05F0E0EE0FD0
:10169000FF1FEE5CFA4F0190F081E02D842F099539
:1016A0000E94A84C8091630081FF06C08091650074
:1016B0008F7E8093650007C0809165008061809374
:1016C00065000E941C078091E00F9091E10F8F71DF
:1016D00090708130910541F082309105A9F08330FE
:1016E000910509F062C050C08091AB0260E00E9499
:1016F0002D08882339F48091490590914A05009777
:1017000009F452C0C79A0895E4EDF0E0E491F0E0E6
:10171000EE0FFF1FED57FA4F8FB7F89420813181FC
:1017200087FF01C07894A90156954795569547952E
:101730008091AA02992787FD9095BC01469FC00120
:10174000479F900D569F900D112443E250E0B90140
:10175000649F9001659F300D749F300D1124820F9E
:10176000931F9695909347058091C405805E809362
:10177000C4058823D1F48091A9029817B0F4809110
:10178000410580933D0508956091BD0270E0687346
:101790007070769567956B527F4F8EE395E044E0CD
:1017A00050E00E9492540895C7980895CF93DF9314
:1017B000EC010E94D14C80E060E1AE0120E00E948B
:1017C000924A82E168E24FE151E00E94C44A82E11C
:1017D00060E340E151E00E94C44A0E94A84C80911D
:1017E000A8020E949E4C8091400580933D050E9476
:1017F000FB4C8823E1F70E94FB4C807F8032D9F7B5
:101800000E94FB4C0E94FB4CFBCFCF93DF93EC017B
:101810000E94D14C82E260E04CE351E020E80E945B
:10182000924A80E068E1AE010E94C44A8CE168E31C
:101830004EE251E00E94C44A0E94A84C8091A80246
:101840000E949E4C8091410580933D050E94FB4C77
:10185000807F8032D9F7DF91CF910895FC0180918C
:101860003C05A82FAF5FA0933C05A53038F08093CE
:101870003C0589EE90E00E94050C089580913E059C
:1018800080933D05B0E0AA0FBB1FAE5CBA4FED934D
:10189000FC938FEB099508951F938091BD0281FD04
:1018A00015C01EE0113131F0812F90E00E947B4D78
:1018B000882321F41F5F1631A9F708C080914105E4
:1018C00080933D058DEF94E30E942E0C1F910895A7
:1018D000E0913C05EE23B1F0882311F0E0E001C077
:1018E000E150E0933C0580913E0580933D05F0E09A
:1018F000EE0FFF1FEE5CFA4F0190F081E02D8EEBB2
:10190000099508958CEF90E00E94050C08950F93BF
:101910001F93CF93DF938091BD0280FD56C08091CD
:10192000E00F9091E10F84319105C8F38091BE02E0
:1019300090E081709070A2E0B0E0A81BB90BEA2F94
:10194000F0E0E353FF4FE491F0E0EE0FFF1FED579F
:10195000FA4F8FB7F8940190F081E02D87FF01C016
:101960007894AA0FBB1FA658BD4F11962D913C919C
:1019700012971F960D911C9150975D96CD91DC9119
:101980005E97C80168E070E00E944254601B710BD2
:10199000620F731F6E177F0724F48091C0028823A3
:1019A00081F02C0F3D1FCE0168E070E00E94425490
:1019B000261B370BE217F30744F48091C0028823FB
:1019C00021F082E491E00E94050CDF91CF911F91FC
:1019D0000F9108958091BD0282FD09C00E94DB45F0
:1019E000883C910520F48FE491E00E94050C089555
:1019F000CF92DF92EF92FF920F931F93CF93DF93DB
:101A00008FEF8ABB1BBA91E897BB9EE798BB9EE31A
:101A100094BB91EC95BB11BA82BB98E092B997EF59
:101A200093B9109261008093620090E190936400FA
:101A3000809365000E94634C0E94BF5380E487B985
:101A400085E886B987E083BF8CE981BF87B783606B
:101A500087BF1FBC8AE08EBD10928B0082E8809306
:101A60008A0080917D00806280937D00789481E17E
:101A70009CE1909333058093320589E10E949E4C4E
:101A80000E9418450E94EA0C0E9488060E94870C5A
:101A90000E944C0C0E9448122DE088E190E00FB6A5
:101AA000F894A89581BD0FBE21BD8AEF95E061E055
:101AB00040E00E945D148091A8020E949E4C87B76E
:101AC000806187BFF0907F05E2B680917F05F816B0
:101AD000C9F7E091C102F0E0EE0FFF1FE050FF4FA9
:101AE0000190F081E02D09950E94CE0A80917E053B
:101AF000833019F4A89510927E0590917F0582B7E6
:101B000020917F059217C9F720E0E901FF24EC2A14
:101B1000FD2A192F00E090E0802B912B2091CC071B
:101B20003091CD078E199F098217930708F4C901D8
:101B30009093CD078093CC07C5CF0F93022F50E031
:101B4000440F551F440F551F47535E4F24E00E941A
:101B50005C4A0F9108950F93022F442319F443EF29
:101B600052E01FC0942F9150242F30E0943090F415
:101B70004091BE0250E0440F551F440F551F415085
:101B80005040420F531F440F551F440F551F4457D9
:101B90005F4F07C0A901440F551F440F551F4E5CEE
:101BA0005D4F24E00E945C4A0F9108950F931F93AC
:101BB000DF93CF9300D0CDB7DEB7382F162F942FF9
:101BC000022F403F69F0442319F0403181F404C0F2
:101BD0008A5F45EC51E007C08A5F41EC51E003C0E9
:101BE0008A5F4DEB51E0202F0E94924A25C0441F8E
:101BF0004427441F405E39839A830E94DA49398121
:101C0000832F8A5F9A81292F332727FD309537FF4D
:101C100003C0309521953F4F332727FD3095215044
:101C20003040A901440F551F420F531F41575E4FCB
:101C3000612F23E00E945C4A0F900F90CF91DF91BB
:101C40001F910F910895EF92FF920F931F93DF93CF
:101C5000CF930F92CDB7DEB7982FE62EF42E1091CA
:101C6000D102412F552747FD509557FF03C050958E
:101C700041955F4F4031ACF483E04802A00111244C
:101C8000425A5E4F892F6E2D23E00F2D99830E94BB
:101C90005C4A99811F3F5CF5892F86506E2D41E289
:101CA00023C04F3174F411161CF4412F4F5002C061
:101CB000412F415F892F86506E2D2F2D0E94D60D0A
:101CC00016C011161CF4412F4E5102C0412F425E26
:101CD000892F86506E2D2F2D99830E94D60D9981C4
:101CE000892F8E5E6E2D4DE62F2D0E94DA490F90C2
:101CF000CF91DF911F910F91FF90EF9008950F9377
:101D00001F93DF93CF930F92CDB7DEB7982F062F97
:101D1000122F442331F4885E46E599830E94DA4904
:101D2000998140914705892F885E602F50E0212FCF
:101D30000E94B34B0F90CF91DF911F910F910895A7
:101D4000DF92EF92FF920F931F93CF93DF93E82ED2
:101D5000F62EEA01122FD02E57FD02C040E201C03C
:101D60004DE28E2D6F2D212F0E94DA4917FD02C002
:101D700081E101C089E1E80E8E2D6F2D4AE3212F0C
:101D80000E94DA49D7FF03C0D095C195DF4FCE013D
:101D90006CE370E00E944254AB01212F2C5F8E2D2A
:101DA0006F2D02E00E94124B17FD02C032E101C00C
:101DB00038E1CE016CE370E00E944254AC012D2D5D
:101DC0002C5F832F8E0D6F2D02E00E94124BDF914E
:101DD000CF911F910F91FF90EF90DF900895282FE2
:101DE00087FD2D5F25952595332727FD30959AE0B2
:101DF0008902C0011124280F391FC90108956F926B
:101E00007F928F929F92AF92BF92CF92DF92EF928A
:101E1000FF920F931F935C01CC24DD243B018824A7
:101E2000992464E670E080E090E0661977098809FB
:101E30009909A60195010E9403547B018C0182E35C
:101E400090E0A0E0B0E0E80EF91E0A1F1B1FC601DB
:101E5000B5010E9403540E940354BC0188279927AE
:101E6000A40193010E94035424E0969587957795E9
:101E700067952A95D1F7E60EF71E081F191FC801AE
:101E8000B70124E630E040E050E00E945554C9011B
:101E90001F910F91FF90EF90DF90CF90BF90AF9088
:101EA0009F908F907F906F900895EF92FF921F9375
:101EB000CF93DF939C016115710521F110E097FF2D
:101EC00004C011E0309521953F4F77FF0EC0C0E070
:101ED000D4E0709561957F4FCE01821B930B0E94D9
:101EE000FF0E9E01281B390B08C0C9010E94FF0E7E
:101EF000E82EE7017E01F92E9701112319F03095A4
:101F000021953F4FC901DF91CF911F91FF90EF9035
:101F10000895E7E0F7E090E02491281711F4892F65
:101F200008953196222311F09F5FF6CF80E0089547
:101F3000883210F080E20895E82FF0E0E95FF84F72
:101F40008491089530E0683008F031E070E0332388
:101F500071F068507040AB01E3E0440F551FEA9503
:101F6000E1F7460F571FBA016C527B4F0AC0AB0115
:101F7000440F551F440F551F460F571FBA01645594
:101F80007B4FFB01208180509C4F97FD0FC0F8E0F4
:101F900080309F078CF0332319F424E030E002C036
:101FA00028E030E0260F371FF9012081332727FD75
:101FB0003095322F222732C0332329F0492F9070D9
:101FC000880F991F03C0492F46959170242F30E048
:101FD000FB01E20FF31F2181332727FD3095AC0170
:101FE00055954795B901649F9001659F300D749F89
:101FF000300D11246081772767FD709540E052E035
:10200000481B590B55954795CA01689FA001699FC8
:10201000500D789F500D1124240F351FC90169E11F
:1020200070E00E944254CB010895CF93DF9320913A
:10203000D602220F285F9091D90284E69802E0012F
:102040001124C85ADD4FEEECF7E0AAEFB5E0422FBD
:1020500050E0440F551F440F551F4E0F5F1F60EB9C
:102060007AE91AC08D919C911197805A964F3DE064
:102070008137930718F080E79DE006C035E0803592
:10208000930710F480E595E0681B790BD183C0833A
:102090009383828334961296E417F50719F7220F7B
:1020A000A22FB0E0AA0FBB1FA253B84F1196DC932A
:1020B000CE932F5F8AE9603B780750F4A22FB0E0FF
:1020C000AA0FBB1FA253B84F11967C936E932F5F3C
:1020D000E22FF0E0EE0FFF1FE253F84F1182108263
:1020E000DF91CF910895A091BE08B091BF08FD0186
:1020F0008193919313967C936E9312973296F093FB
:10210000BF08E093BE080895882329F420EB34E04B
:1021100080EB94E004C020E639E080E699E0A091ED
:10212000BE08B091BF08FD012193319313969C9393
:102130008E9312973296F093BF08E093BE080895ED
:102140001F93182F82700E948410812F81700E942B
:1021500084101F910895CF92DF92EF92FF920F9318
:102160001F93CF93DF938091D5028150833018F075
:10217000FF24F39405C0E82FF0E0E452FE4FF08016
:102180008091FA059091FB0580509C4F880F991F14
:102190002091FC053091FD0520503C4F220F331F4C
:1021A000132F092F97FD00E017FD10E000310CF010
:1021B0000FE010310CF01FE0212F332727FD309561
:1021C000802F992787FD909509968217930714F41D
:1021D000012F0950C02EDD24C7FCD094275F3F4F4C
:1021E0002C153D0514F4102F195080E797E19093BA
:1021F000CF078093CE07C0EBD4E0D093D107C09334
:10220000D00782ED97E09093BF088093BE0880E0EE
:102210000E94A010A091BE08B091BF0880E699E08E
:10222000FD01819391931396DC93CE931297DF0176
:102230001296938382831396DC93CE93129714960F
:10224000B093BF08A093BE088F2D0E94A010F194F8
:10225000C6019595879595958795E82E0E94A010C3
:10226000FE18802F0E94A010F01A812F992787FD59
:1022700090959595879595958795082F0E94A01024
:10228000F01A812F0E94A0108F2D811B0E94A01098
:1022900080E00E948410E091BE08F091BF08DF0149
:1022A000129780E69AEE11969C938E93119211925A
:1022B000F093BF08E093BE08DF91CF911F910F917B
:1022C000FF90EF90DF90CF900895E091BE08F091DD
:1022D000BF08882341F0DF0180E293E08D939D9356
:1022E00080E496E007C0DF0180E496E08D939D9343
:1022F00080E293E0938382831296B093BF08A09309
:10230000BE0808950F931F93082F10E0802F81704F
:102310000E9465111F5F06951830C1F71F910F913C
:1023200008950F931F938EEC97E09093BF088093CE
:10233000BE088091C00891E089278093C008882357
:1023400009F452C00091FA051091FB05085F1B4F7C
:1023500054E0169507955A95E1F70038110510F0ED
:102360000FE710E02091FC053091FD0537FD0FC00F
:10237000C901409645E0969587954A95E1F78034E6
:10238000910510F08FE390E0182F10640FC080E1EA
:1023900090E0821B930B35E0969587953A95E1F78F
:1023A0008034910510F08FE390E0182F802F0E9469
:1023B0008211812F0E948211012710E0C80124E0C0
:1023C000880F991F2A95E1F7B4E015950795BA95FE
:1023D000E1F7802B0E948211A091BE08B091BF0846
:1023E000FD0180E197E231C08091FE059091FF05EB
:1023F00080509C4FA4E096958795AA95E1F7803888
:10240000910510F08FE790E0182F1068812F0E943F
:1024100082118EE80E9482118EE88127282F30E0F9
:10242000C901F4E0880F991FFA95E1F7E4E03595CA
:102430002795EA95E1F7822B0E948211A091BE08B0
:10244000B091BF08FD0180EB96E38193919380EA00
:102450009FE013969C938E9312973296F093BF0849
:10246000E093BE08E091BE08F091BF08119211926E
:10247000F093BF08E093BE08EE5CF740E03FF10543
:1024800024F084EA93E00E94050C1F910F910895B7
:102490008091D502882339F0813068F0843030F0A3
:1024A000843049F406C00E94151008950E94AB10B4
:1024B00008950E9491110895FF920F931F93F82E93
:1024C0001091D102812F992787FD909597FF03C026
:1024D000909581959F4F082F8F31CCF011161CF4E9
:1024E000812F8E5102C0812F825E60E00E942D08F4
:1024F000882359F09091380A992339F42091390AA8
:10250000222309F491E09093390A8093380AE091EC
:102510003C0AF0913D0A3196F0933D0AE0933C0A63
:1025200020913A0A30913B0A2F0D311D30933B0A1E
:1025300020933A0A8091E00F9091E10F40913E0A7A
:1025400050913F0A841B950B8436910508F4F7C01F
:102550004C595F4F50933F0A40933E0AC901BF0157
:102560000E942E54F62E862F90E0AF01849FF0013A
:10257000859FF00D949FF00D11242E1B3F0B30937F
:102580003B0A20933A0A10923D0A10923C0A00310D
:102590001CF41092390A0EC00F3164F411161CF4A9
:1025A000812F8F5002C0812F815F60E00E942D0833
:1025B0008093390A80914107909142070196909348
:1025C00042078093410760914307709144076F5F12
:1025D0007F4F7093440760934307FF2049F0809139
:1025E00047079091480701969093480780934707C3
:1025F0008091390A882349F08091450790914607D8
:1026000001969093460780934507F69440914907B9
:1026100050914A074F0D511D50934A074093490767
:102620008091D3029091D40290934D0780934C07F0
:10263000F091D1022F2F332727FD309537FF03C0AC
:10264000309521953F4F222319F410924B072BC050
:10265000213041F49C01261B370B30934D0720930A
:102660004C0721C02031A0F420FF06C064E056953D
:1026700047956A95E1F704C0409147075091480794
:102680009C01241B350B30934D0720934C070BC046
:102690002091450730914607AC01421B530B5093E4
:1026A0004D0740934C0720914B07222329F02130FE
:1026B00031F02230F9F40EC0FF23E1F018C0209170
:1026C0004C0730914D0712161306A4F0009791F0B5
:1026D00022E00EC020914C0730914D075FEF253C62
:1026E00035071CF423E020934B07009719F421E0F1
:1026F00020934B072091D202222351F020914C07C6
:1027000030914D07821B930B90934D0780934C079C
:1027100080914B07823099F480914C0790914D073E
:102720002091360A3091370A2817390741F09093E3
:10273000370A8093360A8091400580933D051F91AA
:102740000F91FF9008954091D102842F992787FD22
:10275000909597FF03C0909581959F4F982F823059
:1027600094F1803184F585959A3094F4E82FFF2711
:10277000E7FDF0958091BE0290E0880F991F880FC9
:10278000991FE80FF91FE75FFE4F808190E003C0BB
:10279000992787FD90950197FC01EE0FFF1FE753E6
:1027A000FA4F2081318147FF05C080E094E0821B11
:1027B000930B03C0C90180509C4F26E096958795E6
:1027C0002A95E1F702C080E090E00E945C12E0915F
:1027D000BE02F0E0EE0FFF1FEE0FFF1FE45FFE4FA3
:1027E000E081F0E0EE0FFF1FE953FA4F8081918105
:1027F0002091C002222329F020E034E0281B390B6D
:1028000003C09C0120503C4F76E0369527957A9581
:10281000E1F76091320A7091330A6F5F7F4F7093D6
:10282000330A6093320A8091300A9091310A820F04
:10283000931F9093310A8093300A2091E00F3091DA
:10284000E10F4091340A5091350A241B350B43E0C7
:10285000283E340788F12091E00F3091E10F30934A
:10286000350A2093340A1092310A1092300A1092DD
:10287000330A1092320A2091C8073091C9072F5F9E
:102880003F4F3093C9072093C8072091C607309166
:10289000C707F901E25BF84F0E942E5460832F5F57
:1028A0003F4F3093C7072093C6072837310520F0E4
:1028B0001092C7071092C60708952F923F924F9229
:1028C0005F926F927F928F929F92AF92BF92CF92C0
:1028D000DF92EF92FF920F931F93DF93CF93CDB7C9
:1028E000DEB767970FB6F894DEBF0FBECDBF9B8BE8
:1028F0008A8B6C8B4D8780914805882309F474C0BE
:102900008091F905882319F081508093F905409151
:10291000BF02442309F468C08091A4099091A509DD
:10292000A091A609B091A7090196A11DB11D8093A0
:10293000A4099093A509A093A609B093A709809133
:10294000EA099091EB0964E070E00E9442549B0117
:102950008091E8099091E90964E070E00E94425496
:10296000260F371F8091EC099091ED0964E070E02B
:102970000E944254260F371F8091EE099091EF0973
:1029800064E070E00E944254260F371F8091A20934
:102990009091A3092817390761F03093A309209378
:1029A000A2091092A4091092A5091092A6091092EA
:1029B000A709642F70E080E090E02CEB36E140E066
:1029C00050E00E9403542091A4093091A509409140
:1029D000A6095091A709621773078407950720F489
:1029E0008091410580933D057BE7C72E72E0D72E8D
:1029F00068EAA62E64E0B62E54ED452E5FEF552E04
:102A00004A0C5B1C88249924EE24FF24772441E09F
:102A1000242E312C672C7E2C8E2D0E940F069C01BB
:102A2000D6018D919C911197281B390B1216130614
:102A30002CF45C968D919C915D9703C0F601868580
:102A400097858436910514F484E690E0A901662701
:102A500057FD6095762F3AE0440F551F661F771F8C
:102A60003A95D1F749875A876B877C879C01442721
:102A700037FD4095542F69857A858B859C850E940A
:102A80007754022F132F5CEF013015071CF400E080
:102A90001CEF06C064E00030160714F000E014E0FC
:102AA000F401E753FA4F11830083C8010F968F3169
:102AB000910510F574E0E716F104B4F4E091BE025C
:102AC000F0E0EE0FFF1FEE0FFF1FEE0DFF1DE65FA4
:102AD000FE4F808190E00197D10102C0AA0FBB1F79
:102AE0008A95E2F7CD0107C0C1010E2C02C0880F04
:102AF000991F0A94E2F7682AB3E0B71508F4FEC0FC
:102B0000F201808160E00E942D08882311F477246F
:102B10000DC0D20111968C9160E00E942D0888238F
:102B200019F092E0792E02C0772473948091BE024E
:102B300090E081709070E2E0F0E0E81BF90BFA871A
:102B4000E987EE15FF0549F58091D702807F29F1CD
:102B500000501C4FE72DF0E0EE0FFF1FEE0FFF1FA0
:102B6000C701880F991F9C01A3E0220F331FAA956C
:102B7000E1F7281B390BE20FF31FE059FB4F60818F
:102B8000772767FD7095C801959587950E94550F29
:102B9000AC01440F551F30E028C030E0101611067C
:102BA0000CF031E0872D90E0A701440F551FFA018A
:102BB00063E0EE0FFF1F6A95E1F7E41BF50B880F4A
:102BC000991F880F991FE80FF91FEA53FD4FE30F74
:102BD000F11DE655FE4F6081772767FD7095C801AE
:102BE0003F8B0E94550FAC013F89E72DF0E0EE0FBF
:102BF000FF1FEE0FFF1FB701660F771FCB01A3E08A
:102C0000880F991FAA95E1F7861B970BE80FF91F0C
:102C1000EA53FD4FE30FF11DE455FE4F6081772726
:102C200067FD70956C597F4F882777FD8095982FA9
:102C3000DA019D01442737FD4095542F0E9403542B
:102C400024E630E040E050E00E947754022F132F3A
:102C5000E985FA85EE15FF0509F041C08091D7029C
:102C6000982F907F09F4D5C400501440D2C48091AD
:102C7000C002D5012C91882389F0B80160507C4FA7
:102C8000882777FD8095982F332727FD3095432F90
:102C9000532F2D5730404040504011C060E074E049
:102CA000601B710B882777FD8095982F332727FDB0
:102CB0003095432F532F23583F4F4F4F5F4F0E9464
:102CC000035420E038E040E050E00E947754203088
:102CD000B8E03B07B0E04B07B0E05B0729F4F50133
:102CE0002081332727FD3095220F331FE1E0F0E0EC
:102CF000EC0FFD1FE80DF91D31832083F401E8512D
:102D0000F64F118300830894E11CF11C22E030E0AF
:102D1000C20ED31E820E931E0894A11CB11C4EE05D
:102D200050E0440E551E57E0E516F10409F073CE4D
:102D30009091DB0296218091A1098095892321F051
:102D400080913F0580933D059093A10980E094E038
:102D50009093F7098093F6099093F9098093F80905
:102D6000EAEFF9E080E090E09C0123593A4FAC0192
:102D700046585D4FD9012D913C91DA01D2964D9183
:102D80005C91D397241B350B2193319302968031AC
:102D9000910551F798EA492E99E0592EAAE0BAE038
:102DA000F201808191818D939D93349629E0E83ED4
:102DB000F207B9F780914805882311F00E94A31308
:102DC00080E4E8EAF9E0DF011D928A95E9F7BD8524
:102DD000BB23E9F08091BE0290E08170907022E008
:102DE00030E0281B390BA8EEB9E0FE01319680E0F7
:102DF00090E02817390729F011961C921E92118233
:102E000010820196129632968430910591F780EEE9
:102E1000E82E82E0F82E01ECC02E08E0D02E11E45E
:102E2000212E19E0312EE1E8F9E0FA87E9878824BC
:102E300099241D865E8A4D8AB82CA92CD7018C91C5
:102E40008150803108F017C3E985FA8570801082BF
:102E500013968C9161E00E942D08D70111969C91E8
:102E600011978823F9F4892F8850823008F0EAC23C
:102E70009401F901EE0FFF1FA3E0220F331FAA9563
:102E8000E1F7E20FF31FE052FD4F87818E7084302F
:102E900009F4D8C2993019F000E010E038C000E021
:102EA0001CEF35C0E92FF0E0EE0FFF1FEA51F64F9F
:102EB00000811181C401FC01EE0FFF1F53E0880F58
:102EC000991F5A95E1F7E80FF91FE052FD4F8781EE
:102ED000807FE9F0C401FC01EE0FFF1F33E0880F93
:102EE000991F3A95E1F7E80FF91FE951FD4F8081ED
:102EF00082958F7090E00197E1E0F0E002C0EE0F64
:102F0000FF1F8A95E2F7CF01FD85F82BFD8781E051
:102F1000A985BA858C93F7018085882321F00E94CA
:102F2000EF0E080F191F8B2D9A2DFC01EE0FFF1FBE
:102F3000B3E0880F991FBA95E1F7E80FF91FE05247
:102F4000FD4F4680442091F48B2D9A2DFC01EE0F0D
:102F5000FF1F73E0880F991F7A95E1F7E80FF91FBB
:102F6000E052FD4F8581882309F48BC1FC89FF2342
:102F700029F480E0772089F481E00FC0C801AA27F6
:102F800097FDA095BA2FBA2FA92F982F8827F60161
:102F900080839183A283B38380E0D6012D913D91FC
:102FA0004D915C911397882399F4CA01B90120E0EF
:102FB00031E040E050E00E947754509540953095C4
:102FC00021953F4F4F4F5F4F3801620E731E6EC009
:102FD000D701EC91F0E0EE0FFF1FE85FF54F608145
:102FE0007181882777FD8095982F20E034E640E0B6
:102FF00050E00E940354F7012281332727FD3095CA
:10300000432F532F0E947754CA01D6012C93119657
:103010003C93119712964C93129713969C93139787
:10302000B90120E031E040E050E00E947754509533
:103030004095309521953F4F4F4F5F4F3801620EBD
:10304000731E6114710491F177FE10C08B2D9A2DBF
:10305000FC01EE0FFF1F33E0880F991F3A95E1F74F
:10306000E80FF91FEB51FD4F808110C08B2D9A2D79
:10307000FC01EE0FFF1FB3E0880F991FBA95E1F72F
:10308000E80FF91FEB51FD4F808182958F7090E022
:10309000FC0124E630E0E29FC001E39F900DF29F27
:1030A000900D1124D10111969C938E93F101808192
:1030B0009181009771F020914805222319F0019722
:1030C00091838083D6016D917D918D919C91139711
:1030D000D1C06114710409F4D4C0442009F4D1C0F2
:1030E00080914805882309F481C0F70122813327A4
:1030F00027FD3095432F532F60E070E080E293E08E
:103100000E947754B901CA01161417047CF52B2DBF
:103110003A2DF901EE0FFF1F53E0220F331F5A958E
:10312000E1F7E20FF31FEA51FD4F20812F7030E0ED
:103130002115310509F44BC0A901A4E6B0E04A9F6E
:1031400090014B9F300D5A9F300D1124442737FDBD
:103150004095542F0E947754F60180819181A2817D
:10316000B381280F391F4A1F5B1F3AC02B2D3A2D00
:10317000F901EE0FFF1FB3E0220F331FBA95E1F7FD
:10318000E20FF31FEA51FD4F208122952F7030E0AE
:1031900021153105E1F0A901A4E6B0E04A9F9001B4
:1031A0004B9F300D5A9F300D1124442737FD409519
:1031B000542F0E947754DA01C901F6012081318130
:1031C00042815381281B390B4A0B5B0B09C09801C4
:1031D000442737FD4095542F542F432F322F222759
:1031E000D6012D933D934D935C93139798014427FB
:1031F00037FD4095542F2E873F87488B598BD6013A
:103200006D917D918D919C9113971614170484F400
:1032100020E031E040E050E00E9477546E857F85E9
:1032200088899989621773078407950784F01DC000
:1032300020E031E040E050E00E9477548E859F8589
:10324000A889B989281739074A075B0774F4222728
:1032500017FD2095322F322F212F102F0027D60156
:103260000D931D932D933C931397F601608171810B
:103270008281938120E031E040E050E00E94775469
:103280008901D70114966C911497662309F449C0FB
:10329000613059F06230A9F0633029F1643049F1AE
:1032A000653059F1663091F52BC0F7018181893085
:1032B00029F417FD28C0005012400EC017FF31C07E
:1032C0002EC0D70111968C911197893041F41016B8
:1032D000110614F100501E4F000F111F22C01016CE
:1032E0001106ECF01EC017FF1CC0109501951F4F72
:1032F00018C01016110684F012C017FF10C003C0CA
:10330000101611064CF000E01CEF0BC06750C8010E
:103310000E94A20F8C0105C000E014E002C000E092
:1033200010E08B2D9A2DFC01EE0FFF1F63E0880F3C
:10333000991F6A95E1F7E80FF91FE052FD4F878169
:103340008170B1F4D7011196EC911197EE2381F0C1
:10335000E53070F4F0E03197EE0FFF1F21E030E030
:103360002C0F3D1FE20FF31F80819181080F191F61
:10337000B801882777FD8095982FD70112962C9158
:103380001297332727FD3095432F532F0E94035464
:103390002B2D3A2DF901EE0FFF1F03E0220F331FF3
:1033A0000A95E1F7E20FF31FE951FD4F20812695C1
:1033B000277030E02130310589F0D701EC912230BF
:1033C000310569F5F0E0EE0FFF1FEE0FFF1FEC5522
:1033D000F64F608371838283938334C0F701008149
:1033E00010E0000F111F000F111F0C55164F24E69F
:1033F00030E040E050E00E947754CA01B901D801A2
:103400002D913D914D915C9113970E94035420E0C2
:1034100034E040E050E00E947754F8010FC0F0E043
:10342000EE0FFF1FEE0FFF1FEC55F64F208131818D
:1034300042815381260F371F481F591F2083318334
:10344000428353830894811C911C2AE030E0E20EF1
:10345000F31E44E050E0C40ED51E62E070E0260E7C
:10346000371E89859A8501969A87898790E2891601
:10347000910409F0E1CC4D885E888D8580FF0AC0FB
:103480002091E00F3091E10F222321F490913F052C
:1034900090933D0581FF10C02091E00F3091E10F26
:1034A000203431F02091E00F3091E10F283421F4E5
:1034B00090913F0590933D0582FF16C08091E00FEB
:1034C0009091E10F803861F08091E00F9091E10FD1
:1034D000883831F08091E00F9091E10F803921F42C
:1034E00080913F0580933D0560E2C62E64E0D62EB4
:1034F000AA24BB248201D6011196EC901197FF24D7
:10350000E7FCF094E4E6F0E0EE0EFF1E2C9033248E
:1035100027FC30942CE93FEF220E331ED8016D902A
:103520007D908D909C901397611471048104910497
:1035300019F44424552422C016141704180419043D
:1035400044F4B701882777FD8095982FA401930153
:103550000CC0B101882777FD8095982F222733274B
:10356000A90126193709480959090E94035420E185
:1035700037E240E050E00E9477542901C401B301D2
:1035800024E630E040E050E00E947754F8012083C8
:10359000318342835383F501E952FA4F208331830B
:1035A0008E2D0E94EF0E882EE92E822D0E94EF0EA6
:1035B000282D3E2D421653060CF492012817390788
:1035C0000CF49C01D60113968D919C911497820F57
:1035D000931F12962C911297222319F090958195A2
:1035E0009F4FF894EA89FB89EA0DFB1D9183808344
:1035F0007894E5E0F0E0CE0EDF1E0C5F1F4F22E076
:1036000030E0A20EB31E30E2A316B10409F073CF6E
:1036100004C08F7009F02BCB62CB67960FB6F8947D
:10362000DEBF0FBECDBFCF91DF911F910F91FF90F5
:10363000EF90DF90CF90BF90AF909F908F907F9052
:103640006F905F904F903F902F9008950F931F932E
:10365000CF93DF9386E291E0EAE1F6E0DF019C019F
:103660001D9221503040E1F730914007A0EEB2E0CA
:1036700040E081E090E050E06C91662311F420E19D
:1036800001C0262F521740F5182F792F352F3F5F95
:10369000E72FF0E0EF01CC0FDD1FCE0FDF1FFE01A3
:1036A000EE0FFF1FE65EF94F31830081016000835A
:1036B000CC0FDD1FC45ED94F18831F5F44837F5F2B
:1036C000321728F3752F7095382F351B970F920FEF
:1036D000320F832F8150522F662399F1E92FF0E0AA
:1036E000EF01CC0FDD1FCE0FDF1FFE01EE0FFF1F1E
:1036F000E65EF94F21834583208122602083838306
:103700008F5F1A962C911A972196621739F4CC0F75
:10371000DD1FC65ED94F1882148209C0CC0FDD1F91
:10372000C65ED94F88838F5F242F2F5F2483382F65
:103730004F5F1A96403219F48093400704C09F5F90
:103740009BCF30934007DF91CF911F910F91089548
:10375000EF92FF920F931F93DF93CF93CDB7DEB716
:10376000A0970FB6F894DEBF0FBECDBF8E010F5FDE
:103770001F4FC80160E041E00E945D14E2E2F4E006
:103780008AEFE82E85E0F82E418152816081D801D0
:103790002D913C91D7018D919C911197662329F031
:1037A000B901681B790BCB0102C0821B930B840FFC
:1037B000951F9283818335960E5F1F4F82E090E0C4
:1037C000E80EF91E94E0E237F907F1F62091BE0207
:1037D00030E02170307082E090E0821B930B1092F9
:1037E000A8048130910511F01092A904823091054E
:1037F00011F01092AA041092AB0482E00E9462437E
:1038000080913F0580933D05A0960FB6F894DEBFEA
:103810000FBECDBFCF91DF911F910F91FF90EF9021
:1038200008958F929F92AF92BF92CF92DF92EF92C4
:10383000FF920F931F93DF93CF930F92CDB7DEB715
:10384000823209F461C0833209F454C0813609F42C
:1038500076C08436F1F0853699F18038A1F0813850
:1038600009F475C0823809F462C0833809F459C07C
:103870008438F1F08538C1F18E3B09F47FC08F3B6D
:1038800009F095C088C00E94F4050E942E0C80E8C3
:1038900014C084E60E94084E823009F011C680915F
:1038A0002D0A90912E0A0097C1F40AC681E019C032
:1038B00086E497E30E942E0C84E80E94F74D77C0BF
:1038C00085E60E94084E823009F000C680912B0ADE
:1038D00090912C0A009709F4F9C50E942E0C67C03C
:1038E000815080932F0A45C08CEC91E30E942E0CEE
:1038F00085E8E3CF8091BC028F5F8093BC02833068
:1039000060F01092BC0209C08091BC02882311F0C3
:10391000815001C082E08093BC0281E00E9462433A
:1039200028C08AE792E20E94FE0583E8C6CF0E9483
:10393000DD5385E293E20E94FE0582E8BECF8091CE
:103940004B078230A1F583E080934B0712C01092A1
:103950004B071092440710924307109248071092A9
:103960004707109246071092450710924A07109297
:10397000490780913E0580933D0519C080912F0A2B
:10398000082F10E00E94F405F801EE0FFF1FE55D1F
:10399000F54F9183808381E00E94F74D83E00E9480
:1039A000F74D82E00E94F74D81E080932A0A8091D2
:1039B000DA0260E00E942D08882331F080912A0A03
:1039C000882311F40E94A81B8091DA0260E00E9413
:1039D0002D0880932A0A909147058091A902981793
:1039E00010F000E801C002E8E6ECEE2EE2E0FE2E68
:1039F0001AE0812F60E0D7014D917D0120E80E94FF
:103A0000DA49155F1837A9F786E060E141E0202F19
:103A10000E947F0E84E268E146E520E00E94DA49D8
:103A200020914705822F6AE00E94225492509230E2
:103A300010F413E001C012E0822F6AE00E942254C9
:103A40000E9422549150923010F00CE002C01F5F8F
:103A50000BE0045F802F6CE1412F0E94E94B802F27
:103A60006DE1412F0E94E94B80914B07882399F02B
:103A7000823011F000E801C002E840914C075091FB
:103A80004D0782E460E1202F0E94A00E83E368E1ED
:103A900040E00E94230E4091D80213E04102A001B1
:103AA0001124465E5B4F84E260E123E000E00E9467
:103AB0005C4A4091D7024295407F45954595459592
:103AC00045954102A00111244D5E5B4F89E360E101
:103AD00023E00E945C4ACC24DD247FE1E72EF6013E
:103AE000E25EFE4F1081F601E855FB4F008107FDB5
:103AF0000D5F05950595043E0CF404EE0D310CF0B8
:103B00000CE1F601E65EFE4F80818823F9F0812FFB
:103B100064E046E30E94ED4B8091BE0290E08C256C
:103B20009D2580FD04C08091D7028F7061F4812FA4
:103B300081506EE143E00E94ED4B812F8F5F6EE17B
:103B400043E00E94ED4B9E2D901B14C0812F8B51A2
:103B50006CE346E30E94E94BF12EFA948F2D6BE360
:103B600043E00E94E94B8F2D6DE343E00E94E94B57
:103B7000100F9CE36DEFF62EF10E092F03508F2DE1
:103B8000602F47E099830E94ED4B9981692F6D5F0B
:103B90008F2D47E00E94E94B812F8D5F602F47E01A
:103BA0000E94ED4B8F2D602F47E00E94E94B089457
:103BB000C11CD11CB4E0CB16D10409F090CF809188
:103BC000BC02823009F4A1C05AEF852E55E0952E33
:103BD00000E04BE1F42E39E1C32ED12CD401ED915C
:103BE000FC9111978091BC02882321F0813009F06B
:103BF00083C023C0302F33703F9D302D1124202FE0
:103C000026952695220F220F220F285DCF0160E214
:103C100070E00E9442545B01CF0160E870E00E94B6
:103C20004254AB014A195B094E0F5F1F832F8F5D12
:103C3000622F20E20E94B34B5FC0043018F02CE5E5
:103C4000E22E02C094E2E92E802F8370182F110F0C
:103C5000110F180F1A5DCF0160E470E00E9442540A
:103C60005B01CF0162E070E00E9442549B012A197F
:103C70003B09CF0160E071E00E944254260F371FDC
:103C800037FF03C0309521953F4FF901EC9D90011E
:103C9000ED9D300DFC9D300D1124245D3E4F232FF2
:103CA000330F330B2595B22EF9E1F21714F4B9E175
:103CB000BB2E8E2D8951612F43E325E50E94BD4B1C
:103CC000612F62508E2D45E00E94ED4BD4018D9105
:103CD0009C9111971816190614F4E39401C0EB187F
:103CE000612F6F5F8E2D4B2D0E94E94B612F61502C
:103CF0008E2D4B2D0E94E94B0F5FE2E0F0E08E0E1F
:103D00009F1E083009F06ACFE7C38FE161E247E107
:103D10000E94ED4B8FE167E347E10E94E94B85E3A9
:103D200061E247E10E94ED4B8FE161E247E10E94D1
:103D3000E94B8BE461E247E10E94ED4B8BE467E3E2
:103D400047E10E94E94B81E661E247E10E94ED4BC9
:103D50008BE461E247E10E94E94B8AE26BE243E0D7
:103D60000E94ED4B89E26CE243E00E94E94B86E55C
:103D70006BE243E00E94ED4B85E56CE243E00E947C
:103D8000E94B8091C9059091CA05880F991F9C0144
:103D9000F3E0220F331FFA95E1F7820F931F60E0E3
:103DA00078E00E944254262F8091CB059091CC055B
:103DB000880F991FAC0173E0440F551F7A95E1F706
:103DC000840F951F60E078E00E94425470956195E1
:103DD0007F4F665D822F885D45E00E94ED4B8091AC
:103DE000C9059091CA05880F991F9C0153E0220FC5
:103DF000331F5A95E1F7820F931F60E078E00E942D
:103E00004254262F8091CB059091CC05880F991FA5
:103E1000AC0133E0440F551F3A95E1F7840F951F2D
:103E200060E078E00E944254709561957F4F625D3A
:103E3000822F885D45E00E94E94B8091C9059091F1
:103E4000CA05880F991F9C0103E0220F331F0A95B2
:103E5000E1F7820F931F60E078E00E944254262F22
:103E60008091CB059091CC05880F991FAC01B3E0F0
:103E7000440F551FBA95E1F7840F951F60E078E075
:103E80000E944254709561957F4F665D822F845DDC
:103E900045E00E94ED4B8091C9059091CA05880FBD
:103EA000991F9C01F3E0220F331FFA95E1F7820F6F
:103EB000931F60E078E00E944254262F8091CB054A
:103EC0009091CC05880F991FAC0173E0440F551FEA
:103ED0007A95E1F7840F951F60E078E00E944254E4
:103EE000709561957F4F665D822F885D45E00E94E9
:103EF000E94B8091CF059091D005880F991F9C01C7
:103F000053E0220F331F5A95E1F7820F931F60E0B1
:103F100078E00E944254262F8091CD059091CE05E5
:103F2000880F991FAC0133E0440F551F3A95E1F714
:103F3000840F951F60E078E00E944254709561956F
:103F40007F4F665D822F8C5A45E00E94ED4B809139
:103F5000CF059091D005880F991F9C0103E0220F97
:103F6000331F0A95E1F7820F931F60E078E00E940B
:103F70004254262F8091CD059091CE05880F991F30
:103F8000AC01B3E0440F551FBA95E1F7840F951FBC
:103F900060E078E00E944254709561957F4F625DC9
:103FA000822F8C5A45E00E94E94B8091CF05909179
:103FB000D005880F991F9C01F3E0220F331FFA955B
:103FC000E1F7820F931F60E078E00E944254262FB1
:103FD0008091CD059091CE05880F991FAC0173E0BB
:103FE000440F551F7A95E1F7840F951F60E078E044
:103FF0000E944254709561957F4F665D822F885A6A
:1040000045E00E94ED4B8091CF059091D005880F3F
:10401000991F9C0153E0220F331F5A95E1F7820F3D
:10402000931F60E078E00E944254262F8091CD05D6
:104030009091CE05880F991FAC0133E0440F551FB6
:104040003A95E1F7840F951F60E078E00E944254B2
:10405000709561957F4F665D822F8C5A45E00E9476
:10406000E94B6091D1057091D205882777FD809545
:10407000982F26E130E040E050E00E9403547B019D
:104080008C0180E098E5A0E0B0E0E80EF91E0A1F80
:104090001B1FC801B70120E038E040E050E00E945B
:1040A000775450954095309521953F4F4F4F5F4F36
:1040B00097E3D92ED20EC801B70120E038E040E0E6
:1040C00050E00E9477542F5F8AE36D2D422F0E94AB
:1040D000ED4B6091D1057091D205882777FD8095D1
:1040E000982F26E130E040E050E00E9403547B012D
:1040F0008C0180E098E5A0E0B0E0E80EF91E0A1F10
:104100001B1FC801B70120E038E040E050E00E94EA
:10411000775450954095309521953F4F4F4F5F4FC5
:1041200087E3D82ED20EC801B70120E038E040E086
:1041300050E00E9477542F5F8BE36D2D422F0E9439
:10414000ED4B6091D1057091D205882777FD809560
:10415000982F26E130E040E050E00E9403547B01BC
:104160008C0180E098E5A0E0B0E0E80EF91E0A1F9F
:104170001B1FC801B70120E038E040E050E00E947A
:10418000775450954095309521953F4F4F4F5F4F55
:10419000B7E3DB2ED20EC801B70120E038E040E0E3
:1041A00050E00E9477542F5F8CE36D2D422F0E94C8
:1041B000ED4B6091D3057091D405882777FD8095EC
:1041C000982F26E130E040E050E00E9403547B014C
:1041D0008C0180E098E5A0E0B0E0E80EF91E0A1F2F
:1041E0001B1FC801B70120E038E040E050E00E940A
:1041F000775450954095309521953F4F4F4F5F4FE5
:10420000A7E3DA2ED20EC801B70120E038E040E083
:1042100050E00E9477542F5F8FE36D2D422F0E9454
:10422000ED4B6091D3057091D405882777FD80957B
:10423000982F26E130E040E050E00E9403547B01DB
:104240008C0180E098E5A0E0B0E0E80EF91E0A1FBE
:104250001B1FC801B70120E038E040E050E00E9499
:10426000775450954095309521953F4F4F4F5F4F74
:10427000F7E3DF2ED20EC801B70120E038E040E0BE
:1042800050E00E9477542F5F80E46D2D422F0E94F2
:10429000ED4B6091D3057091D405882777FD80950B
:1042A000982F26E130E040E050E00E9403547B016B
:1042B0008C0180E098E5A0E0B0E0E80EF91E0A1F4E
:1042C0001B1FC801B70120E038E040E050E00E9429
:1042D000775450954095309521953F4F4F4F5F4F04
:1042E000E7E3DE2ED20EC801B70120E038E040E05F
:1042F00050E00E9477542F5F81E46D2D422F0E9481
:10430000ED4B6091D5057091D605882777FD809596
:10431000982F26E130E040E050E00E9403547B01FA
:104320008C0180E098E5A0E0B0E0E80EF91E0A1FDD
:104330001B1FC801B70120E038E040E050E00E94B8
:10434000775450954095309521953F4F4F4F5F4F93
:1043500077E3D72ED20EC801B70120E038E040E065
:1043600050E00E9477542F5F84E46D2D422F0E940D
:10437000ED4B6091D5057091D605882777FD809526
:10438000982F26E130E040E050E00E9403547B018A
:104390008C0180E098E5A0E0B0E0E80EF91E0A1F6D
:1043A0001B1FC801B70120E038E040E050E00E9448
:1043B000775450954095309521953F4F4F4F5F4F23
:1043C00067E3D62ED20EC801B70120E038E040E006
:1043D00050E00E9477542F5F85E46D2D422F0E949C
:1043E000ED4B6091D5057091D605882777FD8095B6
:1043F000982F26E130E040E050E00E9403547B011A
:104400008C0180E098E5A0E0B0E0E80EF91E0A1FFC
:104410001B1FC801B70120E038E040E050E00E94D7
:10442000775450954095309521953F4F4F4F5F4FB2
:1044300057E3D52ED20EC801B70120E038E040E0A6
:1044400050E00E9477542F5F86E46D2D422F0E942A
:10445000ED4B45EEC42E43E0D42E30E2F32E11E0B6
:10446000812F60E00E942D08082F8AE06F2DA601A1
:1044700023E00E945C4A1F5F98E0F90EA3E0B0E0E1
:10448000CA0EDB1E143061F729ECC22E23E0D22EB7
:1044900090E3F92E17E0812F60E00E942D08082F8D
:1044A00085E66F2DA60123E00E945C4A1F5FB8EFEE
:1044B000FB0EE3E0F0E0CE0EDF1E1A3061F70CC019
:1044C00080912F0A882309F4F1C971CA80912F0ABB
:1044D000882309F005CA6BCA0F90CF91DF911F9115
:1044E0000F91FF90EF90DF90CF90BF90AF909F9093
:1044F0008F9008950F931F93CF93DF93182F80E031
:1045000060E04EE354E021E00E94924A113658F0F8
:10451000133628F0133639F48AEA93E202C081E1B7
:104520009CE10E94FE0586E068E04AE354E00E94B8
:10453000C44A409143075091440788E168E020E075
:1045400000E00E94A00E86E668E046E354E00E9488
:10455000C44A40914507509146078CE368E020E04B
:104560000E94A00E86E060E142E354E00E94C44A4B
:10457000409147075091480788E160E120E00E94A0
:10458000A00E86E660E14EE254E00E94C44A4091EB
:10459000490750914A07B4E056954795BA95E1F717
:1045A0008CE360E120E00E94A00E86E660E04AE233
:1045B00054E00E94C44A40914107509142078CE365
:1045C00060E020E00E94A00E8091C8079091C9078A
:1045D0008937910518F4C0E0D0E004C0C091C60747
:1045E000D091C70782E06CE34EE70E94E94B85E07B
:1045F0006CE143E20E94ED4B1BE0812F6BE343E053
:104600000E94ED4B1A5F1338C1F716E00CE3FE0170
:10461000E25BF84F4081602F641B812F0E94ED4BBD
:104620002196C837D10510F0C0E0D0E08091C607D0
:104630009091C707C817D90719F01F5F1E3739F7C0
:10464000DF91CF911F910F9108951F93CF93DF9327
:10465000182F80E060E043E454E021E00E94924A99
:10466000113631F40E94DA5381E19CE10E94FE058B
:10467000C4EEDFE01CE0812F68E1488120E10E9468
:10468000DA49812F60E2488920E10E94DA492196C7
:104690001A5F1C3681F780910410882309F456C0F4
:1046A0000E94D85383E090E00E947B4D882351F014
:1046B0008091780290917902807D90709093790238
:1046C0008093780282E090E00E947B4D882351F035
:1046D0008091780290917902807B9070909379021A
:1046E0008093780285E090E00E947B4D882351F012
:1046F00080917802909179028077907090937902FE
:104700008093780284E090E00E947B4D882351F0F2
:104710008091780290917902807E907090937902D6
:10472000809378021092041080917802909179021F
:104730000E94E05380EA9FE00197F1F70E94D65370
:1047400080EF90E09093790280937802DF91CF918F
:104750001F9108951F93182F80E060E040E954E016
:1047600021E00E94924A103639F01136D9F0123603
:10477000B1F01336D9F416C08FEF97E0909309018A
:10478000809308011092CB071092CA071092CD07B0
:104790001092CC0780913E0580933D0507C08AE7C3
:1047A00092E202C081E19CE10E94FE0580E068E0A7
:1047B0004EE754E00E94C44A4091CA075091CB078B
:1047C0005695479584E568E00E94B94B80E060E12A
:1047D0004CE654E00E94C44A4091080150910901FE
:1047E0005695479584E560E10E94B94B80E068E109
:1047F0004AE554E00E94C44A4091CA075091CB0751
:104800008091080190910901481B590B56954795D5
:1048100084E568E10E94B94B80E060E248E454E03E
:104820000E94C44A4091CC075091CD0784E690E0A5
:104830009A01289FA001299F500D389F500D1124E7
:1048400014E0569547951A95E1F784E560E220E477
:104850000E94B34B1F9108956F927F928F92AF92F7
:10486000BF92CF92DF92EF92FF920F931F93DF934D
:10487000CF93CDB7DEB7182F962FD42EF22E802FE0
:104880006E2D222311F420E007C0442311F421E00F
:1048900001C022E0911121E093E6A91631F54C2DDB
:1048A00050E0440F551FFA0133E0EE0FFF1F3A9519
:1048B000E1F7E41BF50BE458FB4F40810E94D60D55
:1048C000FF2009F4AFC0DD2009F4ACC08C2D90E0CE
:1048D000880F991FBC0103E0660F771F0A95E1F767
:1048E000681B790B64587B4F28C092E6A91659F5CE
:1048F0004C2D50E0440F551FFA01A3E0EE0FFF1FAF
:10490000AA95E1F7E41BF50BE358FB4F40810E94A9
:10491000D60DFF2009F486C0DD2009F483C08C2D5C
:1049200090E0880F991FBC01E3E0660F771FEA95BE
:10493000E1F7681B790B63587B4F812F40EF5FEFE6
:1049400020E130E06CC0BB24688877248820D1F552
:104950004C2D50E0440F551FFA0133E0EE0FFF1FBE
:104960003A95E1F7E41BF50BAA0CBB1CAA0CBB1C87
:10497000EA0DFB1DE60DF71DE059FB4F4081552761
:1049800047FD50950E94B34BFF2009F44BC0DD203A
:1049900009F448C08C2D90E0880F991FBC01B3E04A
:1049A000660F771FBA95E1F7681B790B6A0D7B1DBF
:1049B000660D771D60597B4F812F4CE95FEF24E630
:1049C00030E02DC0EC2DF0E0AA0CBB1CAF0173E071
:1049D000440F551F7A95E1F74E1B5F0BA40EB51ED1
:1049E000A80CB11CAA0CBB1CF501E60DF71DE05983
:1049F000FB4F4081552747FD50954C595F4F0E9412
:104A0000B34BFF2079F0DD2069F0B3016A0D7B1D07
:104A100060597B4F812F4CE95FEF20E030E002E0EE
:104A20000E94F008CF91DF911F910F91FF90EF90BE
:104A3000DF90CF90BF90AF908F907F906F90089550
:104A4000EF92FF920F931F93CF93DF93282F30E0C5
:104A5000E901CC0FDD1FC90143E0880F991F4A957A
:104A6000E1F7C80FD91F8E01065E1F4F86ECE82EB6
:104A700082E0F82E0E0D1F1DA9014F5F5F4FCA0186
:104A8000880F991FA3E0440F551FAA95E1F7840FE3
:104A9000951F4A9620953095205E3F4FA901440FFF
:104AA000551FE3E0220F331FEA95E1F7420F531F32
:104AB0008E0D9F1DB8010E94A2548AE0F801119248
:104AC0008A95E9F78091AF0ACE0DDF1D8A8F8B8F13
:104AD00084E68C8F82E00E946243DF91CF911F9128
:104AE0000F91FF90EF900895E82FF0E09F01220FC3
:104AF000331FCF0143E0880F991F4A95E1F7280F34
:104B0000391F265E3F4F86EC92E0AF014F5F5F4F4B
:104B1000BA01660F771FA3E0440F551FAA95E1F76E
:104B2000640F751F665E7F4F680F791FE095F095E3
:104B3000B096AF01440F551FA3E0EE0FFF1FAA95DB
:104B4000E1F74E0F5F1F820F931F0E94A2548AE06D
:104B5000E6E1F4E0DF011D928A95E9F782E00E9428
:104B600062430895EF92FF921F93DF93CF93CDB7E7
:104B7000DEB764970FB6F894DEBF0FBECDBF962F99
:104B8000813208F0A4C0882319F4442341F49FC063
:104B9000803219F4442331F09AC0442319F0182FBD
:104BA0001F5F02C0182F1150A82FB0E09D01220FE7
:104BB000331FBD0153E0660F771F5A95E1F7260FAB
:104BC000371F86ECE82E82E0F82EE20EF31EF70186
:104BD000528D852F8150803108F079C0612F70E0AF
:104BE000FB01EE0FFF1F660F771F660F771F660F23
:104BF000771FE60FF71FEA53FD4FE28DE13108F012
:104C000066C0B90160527D4F992309F19D012F5F64
:104C10003F4FC901880F991F13E0220F331F1A95C8
:104C2000E1F7820F931F9D0120953095205E3F4F45
:104C3000A901440F551FA3E0220F331FAA95E1F7E6
:104C4000420F531F80529D4F0E94A25440C0E5174F
:104C500059F0442331F05031D0F55F5FF701528FA6
:104C600036C0F701828F33C0412F50E0CA01880F50
:104C7000991FE3E0440F551FEA95E1F7840F951F54
:104C800080529D4FDE011B96F901E052FD4F2AE054
:104C900001900D922150E1F7DE011196FE013B9645
:104CA0002AE001900D922150E1F7DB01FC012AE09E
:104CB00001900D922150E1F7DC01FE0131969AE05E
:104CC00001900D929150E1F782E00E946243649658
:104CD0000FB6F894DEBF0FBECDBFCF91DF911F910D
:104CE000FF90EF9008958F929F92AF92BF92CF92D4
:104CF000DF92EF92FF920F931F93CF93DF93EC011C
:104D0000162F49012115310509F43FC0DD248881A2
:104D1000882311F4DD24D394B42EBA94DD2009F154
:104D2000143671F01536E9F4BB20D9F0EB2DF0E024
:104D30003197EE0FFF1FE80DF91D859194910FC07B
:104D4000EB2DF0E0802F90E00197E817F9074CF485
:104D50003196EE0FFF1FE80DF91D859194910E9489
:104D6000FE05402F405D8AE760E02D2D0E94DA4964
:104D700084E760E04FE22D2D0E94DA494B2D4F5C15
:104D80008EE660E02D2D0E94DA49E114F10411F461
:104D900080E009C088818C1508F4C82EF701EC0D5D
:104DA000F11D849181501132E9F0123409F455C09B
:104DB000133409F460C0143461F11534E1F1123692
:104DC00009F44EC0133609F459C0143631F11536C2
:104DD000A9F1113829F01F3B09F05EC018825CC0B0
:104DE0001092F8058091F805882319F01092F805C3
:104DF00053C08881882319F08114910421F480E044
:104E00000E94680C49C080913E0580933D0519823F
:104E100030C09981981709F43FC0E114F104E1F121
:104E20009091F8059923C1F59981981710F49F5F27
:104E300010C019822EC09981992371F1E114F104F7
:104E400059F19091F805992339F59981992319F031
:104E5000915099831EC089831CC088818A15E1F016
:104E60008091F8058823C1F488818A1510F48F5F3A
:104E70000DC018820EC08881882371F08091F805DA
:104E8000882351F48881882319F08150888301C0D8
:104E9000A88280E68093E20FDF91CF911F910F915E
:104EA000FF90EF90DF90CF90BF90AF909F908F904A
:104EB0000895AF92CF92DF92EF92FF920F931F93DC
:104EC000DF93CF930F92CDB7DEB7182F80E060E06D
:104ED00043E755E021E00E94924A88E49AE0612F7E
:104EE00043E026E933E007E059E7E52E55E0F52EEB
:104EF000CC24C394AA24A3940E9473268091480AC8
:104F00001F3B11F41092F805FF24813011F4FF24A7
:104F1000F39480E068E14FE655E023E00F2D0E9416
:104F20005C4ACC24DD2490E300E0043018F4892F9F
:104F300068E103C0892F805660E2D601A359BA4FB9
:104F4000F601E658FD4F4D915C9122A933A9421B11
:104F5000530B440F551F20E299830E94B34B0F5F00
:104F60009981985E22E030E0C20ED31E0830E9F647
:104F7000FF2091F0103681F4ACEAB2E0EDE6F5E006
:104F800080E101900D928150E1F781E00E9462433F
:104F900080913E0580933D050F90CF91DF911F9149
:104FA0000F91FF90EF90DF90CF90AF9008956F92A8
:104FB0007F928F929F92AF92BF92CF92DF92EF92A9
:104FC000FF920F931F93DF93CF930F92CDB7DEB76E
:104FD000182F80E060E043EF56E021E00E94924A03
:104FE0004091A70250E04F5F5F4F845F60E025E093
:104FF00002E00E94124B8BE99AE0612F42E026E822
:1050000033E008E0BAEFEB2EB6E0FB2EACE0CA2EA0
:10501000FCE0AF2E0E947326E0909B0A20919C0A30
:10502000D22ED3941E141CF01092F70515C08E2DAD
:10503000992787FD90953091F705831B910988305A
:1050400091051CF08E2D875005C01816190624F006
:105050008E2D81508093F705123408F44EC014341D
:1050600008F445C01434B1F1153439F1103681F02B
:105070001136C9F0123608F440C01436C0F11436A7
:1050800049F11536D1F01F3BC1F51092F80535C036
:10509000E7FC33C080E09091F805992309F481E0A2
:1050A0008093F8052AC08091F805882331F1109289
:1050B000F80581E60E94F74D20C041E0E416E9F4CE
:1050C0004D15D8F48091F8058823B9F0215020932C
:1050D0009C0A13C051E0E51681F489E08D1568F053
:1050E0008091F805882349F0D0929C0A06C08091EF
:1050F000F805882311F410929C0A8091F705882303
:1051000019F0E8E0FE2E5DC080E068E04EEE56E06B
:1051100020E00E94924AE1E0EE1619F080E090E073
:1051200008C080E090E02091F805222311F481E08E
:1051300090E0082F00618CE368E046EC52E02AE042
:105140000E945C4AF1E0EF16D1F58091F8058823C2
:10515000B1F1AD2CBB240894A108B108F501EA53C4
:10516000FD4F80810E94890F682F809145059091A5
:105170004605009741F4123631F0133621F012340F
:1051800011F0133431F4812F40E027E20E940A0A23
:10519000682F683210F040E205C0E62FF0E0E95FCA
:1051A000F84F4491F501EA53FD4F40838D2D880F50
:1051B0008D0D880F8A5C68E021E00E94DA4970E179
:1051C000F72E8091F705823008F089C080E06F2DBE
:1051D00048EE56E020E00E94924A4091D30250915E
:1051E000D40282E0E816B9F4E1E0DE1639F48091E9
:1051F000F805882309F007C321E00EC0F2E0DF16AE
:1052000051F48091F805882319F420E001E005C0ED
:1052100020E002E002C020E000E086E36F2D0E9463
:10522000A00E42E0E41609F058C08091F8058823EA
:1052300039F48091450590914605009709F44DC0D9
:1052400051E0D51629F082E0D81609F046C020C0FA
:105250008091D3029091D4026CE370E00E942E54AE
:10526000812F40E02BE30E940A0A9CE3890290010F
:1052700011248091D3029091D4026CE370E00E94DB
:105280002E54280F391F3093D4022093D30225C007
:105290008091D3029091D4026CE370E00E942E546E
:1052A000082F0E5F812F602F41E02EE30E940A0A33
:1052B000081B802F992787FD90952091D30230916C
:1052C000D402281B390B3093D4022093D30237FF2A
:1052D00004C01092D4021092D302E8E0FE0E809136
:1052E000F7058330F8F480E06F2D40EE56E020E0C3
:1052F0000E94924A00E0F3E0EF1609F401E08CE32B
:105300006F2D402F0E94230E002351F0812F61ED5D
:1053100072E043ED5FEF2DE230E002E00E94F00822
:1053200048E0F40E8091F705843068F580E06F2D39
:1053300049ED56E020E00E94924A90E054E0E516E4
:1053400009F491E04091D2028AE04802A0011124C0
:105350004C53594F8CE36F2D2AE0092F99830E94FB
:105360005C4A9981992349F0812F6091D20240E0F3
:1053700021E00E940A0A8093D20288E0F80EE8E356
:10538000EF1508F442C28091F7058530F0F580E012
:105390006F2D4DEB56E020E00E94924A90E0F5E040
:1053A000EF1609F491E08091D7028295807F859570
:1053B00085958595859543E08402A00111244A5482
:1053C000594F8CE36F2D23E0092F99830E945C4A8B
:1053D00099819923A1F06091D7026295607F6595CC
:1053E000659565956595812F40E021E00E940A0A48
:1053F0008F709091D702907F982B9093D70248E0BE
:10540000F40E58E35F1508F400C28091F70586306A
:10541000D8F580E06F2D4FEA56E020E00E94924AD6
:1054200090E086E0E81609F491E08091D702859536
:1054300085958595859543E08402A0011124485502
:10544000594F8CE36F2D23E0092F99830E945C4A0A
:105450009981992399F06091D70265956595659535
:105460006595812F40E021E00E940A0A8295807FA5
:105470009091D7029F70982B9093D702E8E0FE0E90
:10548000F8E3FF1508F4C1C18091F705873070F586
:1054900080E06F2D4FE956E020E00E94924A90E0B4
:1054A00047E0E41609F491E04091D80286E0480212
:1054B000A00111244058594F8CE36F2D26E0092F8D
:1054C00099830E945C4A9981992351F0812F68ED5C
:1054D00072E040E050E024E030E002E00E94F0089A
:1054E00058E0F50E88E38F1508F48FC18091F70519
:1054F000883028F580E06F2D48E756E020E00E94D4
:10550000924A00E0E8E0EE1609F401E086E36F2D30
:105510004091DA02202F0E94D60D002351F0812FF6
:105520006AED72E040EF5FEF20E130E002E00E94C0
:10553000F008F8E0FF0E48E34F1508F466C18091CB
:10554000F705893008F05BC080E06F2D4FE656E02C
:1055500020E00E94924A9CE366247724AD2CBB2471
:1055600045010894810891088614970429F459E0AC
:10557000E51611F402E00BC02091DB0230E0062CAE
:1055800002C0359527950A94E2F7022F0170A30116
:105590004959594F892F6F2D21E099830E945C4A08
:1055A0000894611C711C99819A5F9636E9F689E02E
:1055B000E816F9F4103631F08091450590914605D2
:1055C0000097B9F0812F0E94F74D1092F8050894CA
:1055D000A108B10821E030E002C0220F331FAA94D5
:1055E000E2F78091DB0282278093DB0282E00E9457
:1055F0006243E8E0FE0EF8E3FF1508F406C180916F
:10560000F7058A3008F09EC080E06F2D41E656E035
:1056100020E00E94924A4091D5025AE0E51659F4E2
:1056200081E0D81641F48091F805882311F401E057
:1056300003C002E001C000E086E0489FA001112401
:105640004E5B594F84E26F2D26E00E945C4A8091A8
:10565000D502882309F041C04091D602EAE0EE1657
:1056600059F4F2E0DF1641F48091F805882311F433
:1056700001E003C002E001C000E0552747FD50955E
:10568000440F551F440F551F435D594F8CE36F2D39
:1056900024E00E945C4A86E66F2D40E256E020E05E
:1056A0000E94924A4091D9025AE0E51659F483E0EB
:1056B000D81641F48091F805882311F421E003C045
:1056C00022E001C020E082E34802A0011124445DF1
:1056D0005E4F86E66F2D0E94B34BEAE0EE1661F551
:1056E0008091F805882331F4809145059091460515
:1056F000009711F1F1E0DF1639F042E0D41651F0D5
:1057000053E0D516C9F40EC0812F65ED72E040E07C
:1057100050E005C0812F66ED72E04EEF5FEF24E0B0
:1057200030E007C0812F69ED72E04CEF5FEF2AE0B7
:1057300030E002E00E94F00888E0F80EE8E3EF15A0
:1057400008F463C08091F7058B3068F580E06F2D19
:1057500046E156E020E00E94924A90E0FBE0EF161E
:1057600009F491E04091DC0283E0489FA0011124FC
:10577000415F594F8CE36F2D23E0092F99830E94DD
:105780005C4A9981992351F0812F6CED72E040E0E1
:1057900050E021E030E002E00E94F00848E0F40E22
:1057A00058E35F1590F18091F7058C3070F580918A
:1057B000F905882311F020E005C020E08CE0E81610
:1057C00009F421E080E06F2D49EF55E00E94924AF4
:1057D000ECE0EE16D1F41038C1F41092F80589E12E
:1057E0008093F90580E80E94F74D8091A7028F5FB2
:1057F0000E94B1488091A7020E94FD4486E497E38D
:105800000E94FE0502C022E007CD0F90CF91DF91EC
:105810001F910F91FF90EF90DF90CF90BF90AF90CE
:105820009F908F907F906F9008952F923F924F920C
:105830005F926F927F928F929F92AF92BF92CF9220
:10584000DF92EF92FF920F931F93DF93CF93CDB729
:10585000DEB72B970FB6F894DEBF0FBECDBFD82EA4
:1058600080E060E040E457E021E00E94924A84EA50
:105870009AE06D2D43E026E833E008E078E4E72E77
:1058800077E0F72ECC24C39454E0A52E0E94732613
:105890002090A40A2A945090A50A20E6D21661F01E
:1058A00031E6D316A1F080E8D816D9F09FEBD916CF
:1058B00001F51092F8051DC027FC1BC080E09091F7
:1058C000F805992309F481E08093F80512C08091CE
:1058D000F805882371F01092F80581E60E94F74DD3
:1058E00008C027FC06C020929F0A8CE498E30E941F
:1058F0002E0C85E168E040E357E00E94C44AECE7E3
:10590000F4E0FA83E98310EA612E1AE0712E29ECA3
:1059100035E03E832D8310E140E050E0332427FC46
:105920003094C101880F991FFC01A3E0EE0FFF1F07
:10593000AA95E1F7E81BF90BFC83EB835B874A87A9
:10594000FA84E981FA81808160E00E942D08882331
:1059500011F499240DC0E981FA81818160E00E94EF
:105960002D08882319F0F2E09F2E02C09924939409
:10597000292D30E039872887C901880F991F880FA2
:10598000991F4A855B85440F551F9A0163E0220FDA
:10599000331F6A95E1F7241B350B820F931F8A533F
:1059A0009D4FDC01A355BE4FFC01E455FE4F3C91D9
:1059B0002081321711F020E00CC020E0FC01E555F9
:1059C000FE4F86559E4F3081FC018081381709F4C7
:1059D00021E0ED81FE8180819181AC0197FF04C0BF
:1059E00044275527481B590B4A3151050CF020E03C
:1059F000422E8A3191051CF0F301108207C0FFEF9F
:105A0000873E9F071CF421E0F30120838091BE02B2
:105A100090E081709070E2E0F0E0E81BF90B2A85DD
:105A20003B85E217F30751F48091D702807F31F074
:105A3000F901E056F54F1082442443944F2D4F5FF7
:105A400080E0612F20E00E94AB0DF30180811F8276
:105A5000882311F4F1E0FF839091F805992341F434
:105A6000BB2420914505309146052115310511F0E3
:105A7000BB24B3942A853B852216330611F020E01F
:105A800004C020E0552009F421E00F92EDB7FEB7E5
:105A900081838D2D60E04B2D07E2E12ECF2CA92CC8
:105AA00088240E942C240F902A853B8522163306D9
:105AB00009F5552009F0C6C0BB20E1F04420D1F023
:105AC00068857985660F771F660F771F8B819C81AC
:105AD000680F791F9F81690F711D60597B4F8D2D54
:105AE0004CE95FEF24E630E002E00E94F00802C0DB
:105AF00021E001C020E00F92F3018081EDB7FEB7F5
:105B000081838D2D60E04B2D09E3E12ECF2CA92C54
:105B1000882483940E942C240F902A853B8522168A
:105B2000330609F5581409F092C0BB20E1F0442077
:105B3000D1F068857985660F771F660F771F3F81E3
:105B4000630F711D8B819C81680F791F6E587B4F8D
:105B50008D2D4CE95FEF20E030E002E00E94F0087C
:105B600002C021E001C020E00F92EDB7FEB7118224
:105B70008D2D60E04B2D0FE3E12ECF2C33E6A32ECD
:105B800088240E942C240F902A853B8522163306F8
:105B900011F020E005C020E033E0531609F421E0C5
:105BA0000F92EDB7FEB711828D2D60E04B2D07E50A
:105BB000E12ECF2C92E6A92E88240E942C240F904F
:105BC000F3018081882319F4442031F008C0442077
:105BD00031F48AE34FE705C08BE34EE702C08AE366
:105BE0004DE2612F20E00E94DA49F1E09F1621F09A
:105BF00022E0921649F404C085E7612F4DE407C006
:105C000085E7612F4CE403C085E7612F48E420E07D
:105C10000E94DA498A859B8501969B878A87E9815C
:105C2000FA813E96FA83E983185F0894611C711C1F
:105C30002D813E812E5F3F4F3E832D83103309F02F
:105C40007FCE0AC031E0531609F452CF53CF82E021
:105C5000581609F088CF85CF2B960FB6F894DEBF83
:105C60000FBECDBFCF91DF911F910F91FF90EF90AD
:105C7000DF90CF90BF90AF909F908F907F906F906C
:105C80005F904F903F902F9008959F92AF92BF9258
:105C9000CF92DF92EF92FF920F931F93CF93DF93F8
:105CA000182F80E060E043E059E021E00E94924A32
:105CB0008CEB9AE0612F47E026E833E008E07BE0D8
:105CC000E72E79E0F72ECC24C39456E0A52E0E944F
:105CD00073262091BC0AC22ECA94F090BD0AF39498
:105CE0001C141CF01092F70513C08C2D992787FD0A
:105CF00090953091F705831B91098630910524F02A
:105D000026502093F70504C097FF02C0C092F70504
:105D1000103649F0113691F01F3BC9F41092F70587
:105D20001092F80514C0C7FC12C080E09091F805ED
:105D3000992309F481E08093F80509C08091F80562
:105D4000882329F01092F80581E60E94F74D88E13A
:105D500068E045EF58E00E94C44A30E1E32EDD24BC
:105D6000CC2DDD27C7FDD09527E0C22E8091F70509
:105D70008D0D863009F49EC0A82EBB24CA15DB0504
:105D800011F0992409C08091F805882319F4992409
:105D9000939402C092E0992EA5014F5F5F4F82E17C
:105DA0006E2D24E002E00E94124BF501EE0FFF1F62
:105DB000EA0DFB1DE45EFA4F408181E0F81611F414
:105DC000292D01C020E088E16E2D0E94AB0DF50168
:105DD000EE0FFF1FEA0DFB1DE35EFA4F408182E0EC
:105DE000F81611F4292D01C020E0552747FD5095E4
:105DF00088E46E2D0E94B34BF501EE0FFF1FEA0DF4
:105E0000FB1DE25EFA4F408183E0F81611F4092D84
:105E100001C000E04C9DA00111244F52574F8EE469
:105E20006E2D27E00E945C4A8091F805882331F4AA
:105E300080914505909146050097A9F1992099F127
:105E400081E0F81639F082E0F81689F083E0F81660
:105E500051F51AC0B501660F771F6A0D7B1D645E90
:105E60007A4F812F40E050E021E230E019C0B501C7
:105E7000660F771F6A0D7B1D635E7A4F812F4CE999
:105E80005FEF24E630E00CC0B501660F771F6A0DA6
:105E90007B1D625E7A4F812F40E050E024E030E0CD
:105EA00002E00E94F008D39488E0E80E86E0D8165D
:105EB00009F05CCFDF91CF911F910F91FF90EF9090
:105EC000DF90CF90BF90AF909F9008952F923F9218
:105ED0004F925F926F927F928F929F92AF92BF92FA
:105EE000CF92DF92EF92FF920F931F93DF93CF93A6
:105EF000CDB7DEB72F970FB6F894DEBF0FBECDBF7C
:105F0000182F80E060E044E559E021E00E94924AC9
:105F100084ED9AE0612F45E026E833E008E07BE578
:105F2000E72E79E0F72ECC24C39451E1A52E0E94F0
:105F300073262091D40AD22EDA945090D50A539425
:105F40001D141CF01092F70513C08D2D992787FDA5
:105F500090953091F705831B91098630910524F0C7
:105F600026502093F70504C097FF02C0D092F70592
:105F7000103661F01136A9F01038E9F01F3B09F036
:105F80004AC01092F7051092F80545C0D7FC43C0EF
:105F900080E09091F805992309F481E08093F80559
:105FA0003AC08091F8058823B1F11092F80581E696
:105FB0000E94F74D30C08D2D992787FD9095E09177
:105FC000F7059C012E1B3109F901EE0FFF1FE6506A
:105FD000FA4F2081318141E05416E9F4FC01EE0FC3
:105FE000FF1FEE0FFF1FE80FF91FEE5DFB4F408113
:105FF000442319F0309521953F4FFC01EE0FFF1F10
:10600000EE0FFF1FE80FF91FED5DFB4F318320837B
:1060100082E00E94624388E168E042E459E00E9425
:10602000C44A60E1F62E44248D2D992787FD909572
:106030009E838D83BD2CE12E8091F705840D8031E8
:1060400009F45FC1682F70E09B01220F331F220FFC
:10605000331F260F371FF901ED5DFB4FFC87EB87E0
:10606000A901405E5B4F5A874987F901EF5DFB4FFD
:10607000F887EF8310E02A533D4F4CE5C42E41E0F2
:10608000D42EC20ED31E9DE5292E91E0392E220E6C
:10609000331EAB01440F551F46505A4F5A83498354
:1060A000FB01EC53F54FFC83EB83BAE58B2EB1E09B
:1060B0009B2E820E931EABE56A2EA1E07A2E620E15
:1060C000731E8F5F8D87AB2CC4014B019F878E871A
:1060D0002D813E812815390561F4511651F48091C6
:1060E000F805882319F4BB24B39404C0F2E0BF2E52
:1060F00001C0BB24F6012081222339F0F101408147
:106100005181509541955F4F03C0F101408151810C
:10611000E981FA8180819181841B950B83339105FC
:1061200034F4FFEF8E3C9F072CF431E02327EB8102
:10613000FC812083EB81FC818081882311F44EE770
:1061400001C04FE78BE46F2D20E00E94DA49113047
:10615000C9F01230F1F1133009F46DC0143009F4B4
:106160009AC02D813E812815390511F020E004C028
:1061700020E0552009F421E080E06F2D4D850E943C
:106180009D0DB2C0F101408151812B2D206280E331
:106190006F2D0E94B34BBB2009F4A6C08091F80577
:1061A000882339F48091450590914605009709F4BC
:1061B0009BC08E2D6B857C8548E15CEF28EE33E03B
:1061C00006E00E94F008882309F48EC01092860A27
:1061D0008BC0EE85FF8540814456552747FD50957D
:1061E00088E46F2D2B2D0E94B34BBB2009F47CC09B
:1061F0008091F805882339F48091450590914605F2
:10620000009709F471C0EE85FF85808184568083F4
:106210008E2D69857A8543E85FEF2DE730E002E057
:106220000E94F008882311F01092860AEE85FF85FF
:1062300080818C592EC0F30140814C59552747FD70
:10624000509586E66F2D2B2D0E94B34BBB2009F491
:106250004BC08091F805882339F4809145059091D1
:106260004605009709F440C0F30180818C59808372
:106270008E2D6F81788543E85FEF2DE730E002E0F7
:106280000E94F008882311F01092860AF3018081A1
:106290008456808329C0F601808190E0AC01440FD0
:1062A000551F480F591F455C564F8CE66F2D23E054
:1062B0000B2D0E945C4ABB20B9F08091F805882321
:1062C00031F48091450590914605009769F08E2D37
:1062D000F601608140E021E00E940A0AF601108286
:1062E000882311F021E020831F5F153009F0F0CEE4
:1062F000BA2C439438E0F30E46E0441609F09CCEE5
:1063000021C01E2D00E050E1B51609F401E0809196
:10631000F905882311F4202F01C020E082E16F2DC0
:106320004AE259E00E94924A002361F0103851F489
:106330001092F80589E18093F90580E80E94F74DF5
:106340000E94A81B2F960FB6F894DEBF0FBECDBFDC
:10635000CF91DF911F910F91FF90EF90DF90CF9041
:10636000BF90AF909F908F907F906F905F904F9075
:106370003F902F900895AF92CF92EF92FF920F939C
:10638000AE2CEE24FF24CC240E9473260F91FF90A4
:10639000EF90CF90AF900895DF92EF92FF920F931E
:1063A0001F93DF93CF9300D0CDB7DEB7182F80E0D7
:1063B00060E046E355E021E00E94924A80E49AE0E2
:1063C000612F41E026E933E007E059E0E52E0E9425
:1063D000BB31E090400A1E141CF01092F70515C066
:1063E0008E2D992787FD90952091F705821B9109A5
:1063F000883091051CF08E2D875005C0181619069F
:1064000024F08E2D81508093F7058091F70581301F
:1064100031F482E08E150CF080E08093F7058091D6
:10642000F705882319F048E0F42E25C084E268E0DF
:106430004DE255E00E94C44A00E0E1E0EE1609F4A6
:1064400001E04091A80288E168E050E0202F0E941E
:10645000B34B002371F0812F68EA72E044E150E011
:106460002DE230E001E00E94F0088091A8020E9435
:106470009E4C30E1F32E8091F705823010F588E1D3
:106480006F2D4FE155E00E94C44A4091A902F2E00D
:10649000EF1611F020E201C021E288E16F2D50E0FB
:1064A0000E94B34B82E0E81651F4812F69EA72E052
:1064B00042E350E024E630E001E00E94F008E8E02A
:1064C000FE0E8091F705833008F588E16F2D4DE0D1
:1064D00055E00E94C44A00E0F3E0EF1609F401E041
:1064E0004091BF0288E16F2D50E0202F0E94B34BF6
:1064F000002351F0812F6FEB72E040E050E02AEF73
:1065000030E001E00E94F00888E0F80E8091F70585
:10651000843070F584E26F2D42E055E00E94C44A59
:1065200090E0E4E0EE1609F491E04091C10250E001
:10653000440F551F440F551F4B505B4F80E06F2D8C
:1065400024E0092F9A830E945C4A9A81992351F092
:10655000812F61EC72E040E050E022E030E001E0A9
:106560000E94F008F8E0FF0E88E38F1508F457C189
:106570008091F705853068F584E26F2D48EE54E090
:106580000E94C44A90E0E5E0EE1609F491E04091E3
:10659000C00283E0489FA00111244F515B4F86E069
:1065A0006F2D23E0092F9A830E945C4A9A819923D8
:1065B00051F0812F60EC72E040E050E021E030E0EB
:1065C00001E00E94F008F8E0FF0E88E38F1508F460
:1065D00026C18091F705863020F584E26F2D48EDC5
:1065E00054E00E94C44A00E0E6E0EE1609F401E03F
:1065F00080E06F2D4091AB02202F0E94D60D00232A
:1066000051F0812F6BEA72E040EF5FEF20E130E064
:1066100001E00E94F008F8E0FF0E88E38F1508F40F
:10662000FEC08091F705873008F03FC084E26F2DEF
:1066300048EC54E00E94C44A8091C2028823B1F021
:1066400088E16F2D45EC54E00E94C44A4091C2029B
:1066500085E0489FA001112420E0E7E0EE1609F450
:1066600021E088E16F2D0E94B34B0CC000E0F7E001
:10667000EF1609F401E086E06F2D41EC54E023E0D1
:106680000E945C4A87E0E81651F4812F62EC72E0C8
:1066900040E050E028E730E001E00E94F008E8E048
:1066A000FE0EF7E3FF1508F4BAC08091F7058830B5
:1066B00008F067C084E26F2D43EB54E00E94C44AA7
:1066C000DD2488E0E81611F4DD24D394E091C302C0
:1066D000F0E0EE0FFF1FEE0FFF1FEE5DFE4F40815B
:1066E00050E043555B4F86E06F2D21E00D2D0E9459
:1066F0005C4AE091C302F0E0EE0FFF1FEE0FFF1FB8
:10670000EE5DFE4F418150E049555B4F8CE06F2DAF
:1067100021E00E945C4AE091C302F0E0EE0FFF1F0F
:10672000EE0FFF1FEC5DFE4F408150E04F555B4F79
:1067300082E16F2D21E00E945C4AE091C302F0E00B
:10674000EE0FFF1FEE0FFF1FEE5DFE4F438150E087
:1067500045565B4F88E16F2D21E00E945C4ADD20A9
:1067600051F0812F63EC72E040E050E027E130E02F
:1067700001E00E94F008E8E0FE0EF8E3FF1508F4DF
:106780004EC08091F705893008F049C086E06F2D32
:1067900046E954E020E00E94924A87E38F1590F08A
:1067A00034E290E0832F6F2D4BE353E0292F00E07C
:1067B00039839A830E9469499A819F5F3981385E43
:1067C000943081F7E8E0FE0EF8E3FF1540F1DD2498
:1067D00089E0E81611F4DD24D3944091BE024F5CA9
:1067E00082E16F2D2D2D0E94DA4994E200E00F5FC7
:1067F000892F6F2D402F20E09A830E94AB0D9A8144
:10680000985E0430A1F7DD2051F0812F6EEB72E02D
:1068100040E050E023E030E001E00E94F0080F90FB
:106820000F90CF91DF911F910F91FF90EF90DF902C
:1068300008956F927F928F929F92AF92BF92CF9264
:10684000DF92EF92FF920F931F93CF93DF93182F56
:1068500080E060E044E655E021E00E94924A84E452
:106860009AE0612F42E026E933E007E0A4E0EA2E57
:106870000E94BB316090440A6A94F3E4CF2EF5E0A5
:10688000DF2EE0E1FE2EC0E0D0E0772467FC7094BC
:1068900071E0A72EB12CEE246C167D0611F4EE24C7
:1068A000E3948AE26F2DA60128E000E00E945C4A92
:1068B000C33069F145010C2E02C0880C991C0A9462
:1068C000E2F78091BD02882121F401E040E455E027
:1068D00002C04CE355E082E16F2D2E2D0E94924ABA
:1068E000EE2049F0812F602F40E021E00E94D8097E
:1068F000811181E0082F8091BD0288298093BD021B
:10690000002381F1809488228092BD022BC0809167
:10691000BD028873882E992463E0959487946A95C4
:10692000E1F7082D88E16F2D482D50E02E2D0E94B3
:10693000B34BEE2039F0812F682D40E024E00E9417
:10694000D809082F202F30E00C2E02C0220F331F51
:106950000A94E2F788E380959091BD028923822B07
:106960008093BD02219698E0F90E88E090E0C80E71
:10697000D91E90E3F91609F08ECFDF91CF911F91C8
:106980000F91FF90EF90DF90CF90BF90AF909F90CE
:106990008F907F906F900895EF920F931F93182F11
:1069A00080E060E04BE755E021E00E94924A8CE4F1
:1069B0009AE0612F44E026E933E007E0EE240E94EC
:1069C000BB3180E060E14AE253E00E94C44A80E0CB
:1069D00068E148EF52E00E94C44A80E060E24AE089
:1069E00053E00E94C44A80E068E24BE153E00E9419
:1069F000C44A1F910F91EF900895CF92DF92EF92CA
:106A0000FF920F931F93DF93CF9300D0CDB7DEB7E4
:106A1000182F80E060E04AEA55E021E00E94924AA7
:106A200080E59AE0612F45E026E933E007E0EE24B7
:106A30000E94BB319EE0C92ED12C00E010E0143042
:106A400010F4F02E03C088EFF82EF00EC6010E945D
:106A50007B4DE82E1F5F8AE26F2D412F20E00E94C0
:106A6000D60D4E2D405D84E46F2D2E2D0E94DA4907
:106A7000085F0894C11CD11C193009F71BE8C12E0E
:106A800015E0D12E08E310E0812F90E00E947B4DAD
:106A9000F82E80E0602FA60125E00E948C4A4F2D41
:106AA000405D80E2602F2F2D0E94DA491F5F085061
:106AB00085E090E0C80ED91E163031F784E568E114
:106AC00043E855E027E00E948C4AB6E0EB2EF12C1B
:106AD00010E230E084E5612F4BE353E0232F00E028
:106AE0003A830E946949C7010E947B4D282FC70144
:106AF000019629830E947B4D082F2981422F405DFA
:106B00008CE6612F0E94DA49402F405D88E7612FB3
:106B1000202F0E94DA493A813F5F185FE2E0F0E0FF
:106B2000EE0EFF1E3430B1F60F900F90CF91DF9133
:106B30001F910F91FF90EF90DF90CF900895EF920B
:106B4000FF920F931F93CF93DF93182F80E060E0A5
:106B500040EC55E021E00E94924A84E59AE0612FE2
:106B600046E026E933E007E0EE24E3940E94BB31DF
:106B7000E090540AC0E0D0E000E0FF24AE014155AF
:106B80005A4F88E1602F22E00E948C4A8F2D0E948C
:106B90000F06AC0180E3602F0E94C84A87E0F81618
:106BA000D9F0FE01E753FA4F60817181882777FDA4
:106BB0008095982F24E630E040E050E00E94035496
:106BC00020E034E040E050E00E94775486E6602FF9
:106BD000A9010E94B94B0BC081E0E81611F421E233
:106BE00001C020E28EE4602F40E00E947F0EF3940B
:106BF000085F229688E0F81609F681E0E81651F45D
:106C0000812F6AEA72E041E85FEF2FE730E001E0B0
:106C10000E94F008DF91CF911F910F91FF90EF90AC
:106C20000895AF92BF92CF92DF92EF92FF920F93AF
:106C30001F93CF93DF93182F80E060E041EE55E083
:106C400021E00E94924A82E89AE0612F47E026E91B
:106C500033E007E053E0E52E0E94BB31F090820A5A
:106C6000C6E6DAE038E5A32E3AE0B32E6E0100E086
:106C7000802F0E940F06F60140815181282F392F65
:106C8000421753070CF49A01F60131832083F50172
:106C900020813181821793070CF4C901F50181939A
:106CA00091935F010F5F82E090E0C80ED91E07301C
:106CB000F9F6123261F01F3B09F073C088E99AE3DC
:106CC00089939993EAE0C437DE07D1F76AC0F2E00E
:106CD000FF1629F023E0F21609F063C00CC0C4E7E8
:106CE000DAE010E0812F0E940F06899399931F5FCD
:106CF0001730C1F752C0CBE7D2E0FE0120E030E010
:106D0000D901AA59B54FAD90BC90D901A85AB54F39
:106D1000CD90DC901197C5018C199D0997FF03C098
:106D2000909581959F4F8333910504F1D901AC581B
:106D3000B54F0D911C91119711830083C8018A19D9
:106D40009B095C0160E470E00E944254A61AB70AF5
:106D5000B786A686C601801B910B8C0160E470E0AB
:106D60000E944254061B170B158F048F2E5F3F4F56
:106D700032962E30310521F680E090E0299139914C
:106D8000820F931FE2E0C339DE07C1F79093A6029A
:106D90008093A50281E00E94624380913E0580932A
:106DA0003D052BECC22E25E0D22E10E1C0E0D0E054
:106DB000AF2CBB24A7FCB094219600E0AC16BD0616
:106DC00009F401E080E0612FA60127E00E945C4AFF
:106DD000185F87E090E0C80ED91E183269F7CBE73C
:106DE000D2E0CC24DD2418E000E082E4612F44EC02
:106DF00055E00E94C44A92E0F91631F4F601EA59CE
:106E0000F54F4081518102C04E855F858DE2612F33
:106E10000E94C84AE1E0FE1629F4802F0E940F0666
:106E2000482F0BC0F2E0FF1631F4F601EC58F54F95
:106E30004081918102C04881998188E4612F592F56
:106E40000E94C84A22E0F21631F4F601E85AF54FE2
:106E50004081518102C04C8D5D8D86E6612F0E947C
:106E6000C84A0F5F185F82E090E0C80ED91E2296D4
:106E7000073009F0BACFDF91CF911F910F91FF90AA
:106E8000EF90DF90CF90BF90AF900895CF92DF92B8
:106E9000EF92FF920F931F93CF93DF93182F80E011
:106EA00060E040EF55E021E00E94924A8CE360E010
:106EB0004BEE55E00E94C44A0E94DB45AC018CE6D3
:106EC00060E020E00E94B34B8EE660E047EE55E0C4
:106ED00021E00E94924AF090970A87E99AE0612F98
:106EE00040E020E030E000E07FE0E72E0E94BB3190
:106EF000E090970A1036E1F1113641F01436A1F016
:106F00001038E1F11F3B09F057C04DC08091960A3F
:106F1000882351F01092960A80913E0580933D059A
:106F200081E60E94F74D48C08091A7028E1591F02E
:106F3000812F0E94F74D8091970A8093A7020E94AB
:106F4000FD4481E00E9462431092860A80913E05D2
:106F500080933D05143629F487ED97E20E94FE05E3
:106F60002BC0113649F586E497E30E942E0C24C00D
:106F700081E08093960A80913E0512C08091960A26
:106F80008823D1F08E2D0E94E443882339F080912C
:106F90003E0580933D051092960A0EC080914005F3
:106FA00080933D0509C01092960A8091A7028093B4
:106FB000970A81E00E9472438091960A882341F0EB
:106FC000FE1431F06E2D6F5F8F2D8F5F0E949746FC
:106FD000CE2DDD27C7FDD0958091F7059E01281B9A
:106FE0003109121613065CF0CE01019797FF02C01B
:106FF00080E090E08093F70510E1FF240BC025307E
:107000003105D4F3CE0104978B3091059CF38AE0CF
:1070100090E0F0CFE090F705EF0CCE2CDD24CC15FE
:10702000DD0511F024E001C025E0A6014F5F5F4FB0
:1070300082E1612F02E00E94124B8091A702E816C4
:1070400031F481E0612F4AE220E00E94DA498E2D7E
:1070500067E87AE04FE00E949444CC15DD0531F4F6
:107060008091960A882311F001E101C000E188E1D6
:10707000612F47E85AE02FE00E945C4AF394185FC2
:1070800036E0F31639F6DF91CF911F910F91FF9003
:10709000EF90DF90CF9008952F923F924F925F92A2
:1070A0006F927F928F929F92AF92BF92CF92DF9218
:1070B000EF92FF920F931F93DF93CF93CDB7DEB77D
:1070C00028970FB6F894DEBF0FBECDBF182F80E013
:1070D00060E048E757E021E00E94924A40919F0A11
:1070E0004F5F60E020E00E94AB0D89EA9AE0612FDB
:1070F00040E020E030E000E053E0E52E0E94BB31AC
:10710000D090A90A103611F01F3B11F41092F80527
:1071100080919F0A90E0880F991FFC0133E0EE0FE9
:10712000FF1F3A95E1F7E81BF90BE458FB4F80810C
:1071300060E00E942D08882311F4FF241AC080917A
:107140009F0A90E0880F991FFC0103E0EE0FFF1FDC
:107150000A95E1F7E81BF90BE358FB4F808160E0EB
:107160000E942D08882319F0B2E0FB2E02C0FF24F4
:10717000F39440919F0A642F70E0FB01EE0FFF1F14
:10718000E753FA4F808191818A3191051CF010926A
:10719000A80A07C02FEF873E92071CF481E0809376
:1071A000A80A2091BE0230E02170307082E090E0A9
:1071B000821B930B8617970741F4443030F480917B
:1071C000D702807F11F01092A80A80E060E143E7C7
:1071D00057E00E94C44A0F92EDB7FEB7319620E007
:1071E000DD2009F421E08091A80A8083812F61E0ED
:1071F00041E006E3F0E1EF2EC0909F0AAF2C882417
:107200000E942C240F9080E068E14CE657E00E9439
:10721000C44A0F92EDB7FEB7319620E031E0D316A5
:1072200009F421E08091A80A8083812F61E041E088
:1072300006E3E8E1EE2EC0909F0AAF2C88248394E9
:107240000E942C240F9080E060E246E657E00E9406
:10725000C44A0F92EDB7FEB7319620E042E0D41653
:1072600009F421E01082812F61E041E00EE170E23B
:10727000E72EC0909F0A53E6A52E88240E942C2456
:107280000F9080E068E240E657E00E94C44A0F9207
:10729000EDB7FEB7319620E053E0D51609F421E0B2
:1072A0001082812F61E041E00EE138E2E32EC090D0
:1072B0009F0A92E6A92E88240E942C240F9081E038
:1072C000F81621F092E0F91659F405C080E060E369
:1072D00049E557E009C080E060E342E557E004C0BB
:1072E00080E060E34AE457E00E94C44A40919F0A6C
:1072F000642F70E08F2D90E0880F991F880F991FE1
:10730000FB01EE0FFF1F9F01A3E0220F331FAA9581
:10731000E1F72E1B3F0B820F931F8A539D4FFC01F9
:10732000E655FE4F1081FC01E555FE4F5080FC01F3
:10733000E455FE4F00810C5983559E4FFC01F080AF
:10734000F4E6FF0E2091BE0230E02170307082E042
:1073500090E0821B930B8617970709F058C04430C2
:1073600008F055C08091D702807F09F450C0CC242A
:10737000DD241A821982612E772467FC7094202EF6
:10738000332427FC309450E4852EE980C60196957D
:107390008795B3010E94550F880F991F25E0969598
:1073A00087952A95E1F7BEE3AB2EAE0C9C01229D9A
:1073B000C001239D900D329D900D112464E670E074
:1073C0000E942E54382D361B632F8A2D0E94F44ABA
:1073D00089819A8183709070009751F48A2D6FE3B0
:1073E0000E94F44A6E2D6695605E8EE30E94F44A18
:1073F00049815A814F5F5F4F5A83498380E290E011
:10740000C80ED91E4034510509F0BFCF89C0188677
:107410001F82A0E2DA2EAA24BB24212E332427FCCB
:107420003094E02FFF27E7FDF095FA83E983F0E23F
:107430007F2E852C992487FC90949C828B822F2D03
:10744000332727FD30953E832D836F804884862D1A
:10745000942DB1010E94550FE5E096958795EA9528
:10746000E1F77EE5C72ECA0CAC01E981FA814E9F97
:10747000C0014F9F900D5E9F900D112464E670E057
:107480000E942E54F72DF61B6F2F8C2D0E94F44A6C
:1074900063E0862E912C8A209B208114910449F46C
:1074A0008C2D60E20E94F44A6A2D605E8EE50E9497
:1074B000F44A862D942D6B817C810E94550F55E0F6
:1074C000969587955A95E1F74EE3E42EED0C9C01D5
:1074D0004D815E81249FC001259F900D349F900DAA
:1074E000112464E670E00E942E54605E8E2D0E948E
:1074F000F44A8114910441F48E2D60E20E94F44A12
:107500008EE56D2D0E94F44A0894A11CB11CDA94FA
:107510008F819885809698878F83DD2009F095CF9D
:10752000E0919F0AF0E0EE0FFF1FE753FA4FA080B3
:10753000B180C50125E0969587952A95E1F7825A95
:1075400060E040E40E94ED4B40919F0A2091BE0212
:1075500030E02170307082E090E0821B930B242F8A
:1075600030E08217930709F040C0443008F03DC076
:107570008091D702807FC9F1C50180509C4F62E0A5
:1075800070E00E944254CB01612F772767FD709510
:107590000E94550F07FD0D5F05950595202F332798
:1075A00027FD3095220F331FFC012E9FC0012F9F16
:1075B000900D3E9F900D112469E170E00E944254AD
:1075C0007B01CB01B5E096958795BA95E1F760E42C
:1075D000681B8EE340E40E94E94BC70162E070E063
:1075E0000E944254E62EF72E32C01A141B0414F0E7
:1075F000652D01C0612F772767FD7095C5010E9439
:10760000550F1A141B040CF00F2D07FD0D5F059587
:107610000595202F332727FD30954C01289DC0016B
:10762000299D900D389D900D112469E170E00E9414
:107630004254E62EF72EC701A5E096958795AA95A8
:10764000E1F760E2681B8EE340E40E94E94BF9E158
:10765000CF2ED12CAC9CC001AD9C900DBC9C900D4C
:10766000112460E071E00E944254AB0182E760E3C4
:1076700020E00E94B34BEC9CC001ED9C900DFC9C63
:10768000900D112460E071E00E944254AB0184E54A
:1076900068E020E00E94B34B1A141B045CF4612FD5
:1076A000772767FD7095C50144970E94550FE81A2A
:1076B000F90A0CC0652D772767FD7095C5014496C2
:1076C0000E94550F9C012E193F097901A701440F13
:1076D000551F440F551F4E0D5F1D84E560E124E4E6
:1076E00003E00E94124B28960FB6F894DEBF0FBE3F
:1076F000CDBFCF91DF911F910F91FF90EF90DF9061
:10770000CF90BF90AF909F908F907F906F905F9041
:107710004F903F902F9008954F925F926F927F927B
:107720008F929F92AF92BF92CF92DF92EF92FF9291
:107730000F931F93CF93DF93182F80E060E04AED03
:1077400057E021E00E94924AE0904007EA9483EBE0
:107750009AE0612F44E026E833E008E00E94BB3164
:10776000F090B30AFF2011F41092B20A123491F192
:10777000133471F11036C9F0113609F445C01236D0
:1077800049F1133629F1103809F448C01E3BC9F1FC
:107790001F3B09F053C01092F7051092B10A81E027
:1077A0008093B00A1092B20A2CC01F1444F480E0F7
:1077B0009091B20A992309F481E08093B20A8091F2
:1077C000B20A8093B00A8091AD0A8823B9F123C030
:1077D0001092B00A8091B20A882381F140E01236FB
:1077E00009F441E08091AE0A6091B00A0E94B2258E
:1077F0008091B00A882319F0133609F4FA94109294
:10780000B00A0E94261B1AC08091B20A882319F080
:1078100081E60E94F74D1092B20A10C01F1474F452
:107820008091AD0A882321F08091AE0A0E94202524
:107830001092B20A8AEA9FE30E942E0C84E268E06A
:107840004BEC57E00E94C44AA0E1EA2EDD24DA9412
:10785000F3E67F2ECC2488248A9455245394E3E0C5
:107860004E2E6090F7056C0CC62DD0E0FE01EE0F99
:10787000FF1FEC0FFD1FEE0FFF1FE65EF94F80812B
:10788000982F917021F48695817039F40CC180E0B5
:107890006E2D418120E00E949D0D1F140CF55E01AC
:1078A000AA0CBB1CAC0EBD1EF501EE0FFF1FE45E63
:1078B000F94F8081F816A1F46E2D695F80E048E1F0
:1078C0000E94E94BF501EE0FFF1FE65EF94F848140
:1078D0008093AE0A81818093AF0A5092AD0A8C2CBE
:1078E000FE01EE0FFF1FEC0FFD1FEE0FFF1FE65E08
:1078F000F94F80818695817009F4AAC085812AE0BC
:1079000082025001112480EE92E0A80EB91E992443
:107910008381F81611F499249394F50147814695D3
:1079200047708091B20A882311F0092D01C000E050
:1079300050E04953584F82E16E2D21E00E945C4A8D
:10794000F5014281552747FD50958DE26E2D292D79
:107950000E94B34B8091B20A882311F0292D01C0F7
:1079600020E08DE26E2D45E20E94DA49F501418169
:107970008091B20A882311F0292D01C020E086E30E
:107980006E2D0E94AB0DF5014381442359F0809187
:10799000B20A882311F0292D01C020E08EE46E2D5B
:1079A0000E94D60DF5014481442389F08091B20AEA
:1079B000882311F0092D01C000E0449DA00111248D
:1079C0004F57584F86E66E2D23E00E945C4AF50122
:1079D0008581811181E0F5019681992329F0882321
:1079E00009F491C04AE203C0882361F044E4809125
:1079F000F805882311F0292D01C020E089E76E2DBC
:107A00000E94DA49F1E09F1619F5B5016E5F7F4FCC
:107A1000812F43E85FEF2DE730E002E00E94F0089D
:107A2000FE01EE0FFF1FEC0FFD1FEE0FFF1FE65EC6
:107A3000F94F85818093AE0A81818093AF0A1092BD
:107A4000AD0A8C2C8091B20A882311F46092B10A9D
:107A5000FE01EE0FFF1FEC0FFD1FEE0FFF1FE45E98
:107A6000F94F8081882329F087150CF4782E8D1525
:107A70000CF48D2DFE01EE0FFF1FEC0FFD1FEE0F1E
:107A8000FF1FE65EF94FD380DD2029F0D7140CF4F8
:107A90007D2CD8160CF4D82EC39428E0E20E86E094
:107AA000C81609F0DECEFF20A1F09FEF891689F4F9
:107AB000F71464F48091F70590E00197EFEF8F3FA2
:107AC0009E0711F480E090E08093F705DF14ECF45A
:107AD00014C0F1E0F8155CF08091F70590E0019793
:107AE0002FEF8F3F920761F480E090E009C084E0BF
:107AF00088155CF496E09C1540F48091F7058F5F43
:107B00008093F70502C043E572CFDF91CF911F91BB
:107B10000F91FF90EF90DF90CF90BF90AF909F902C
:107B20008F907F906F905F904F9008956F927F92AB
:107B30008F929F92BF92CF92DF92EF92FF920F931C
:107B40001F93DF93CF9300D0CDB7DEB7182F80E01F
:107B500060E040E659E021E00E94924A88ED9AE018
:107B6000612F46E026E833E008E050E1E52E0E9470
:107B7000BB312091D80AC22ECA941C141CF010925A
:107B8000F70513C08C2D992787FD90953091F70547
:107B9000831B91098730910524F027502093F70526
:107BA00004C097FF02C0C092F705103629F01F3BB2
:107BB00059F41092F70508C0C7FC06C0C092B70A76
:107BC0008EE79EE30E942E0CEE24FF2401E018E0D5
:107BD000DD24C7FCD0949091F7059E0DBB2498300E
:107BE00028F0BB24B394073020F071C0083008F0AF
:107BF0006EC0892E992430E0C814D90409F431E00C
:107C0000FF2019F0FF24F39401C0F32E80E0612FD0
:107C10004DE559E0232F39839A830E94924A9A8135
:107C20003981993010F087E101C082E1A4014F5FF2
:107C30005F4F612F232F0E94B34BBB2071F0940143
:107C400028503040C90143E0880F991F4A95E1F759
:107C5000820F931F8C529B4F09C0C401880F991F3C
:107C6000880F991F880D991D84559B4F3C014C012D
:107C70009AE2F40141914F01552747FD5095892F14
:107C8000612F20E09A830E94B34B9A819B5E9339C7
:107C900081F7185F0F5FBB20A9F09AE2F3014581DD
:107CA000552747FD5095892F612F20E09A830E9428
:107CB000B34B0894611C711C9A819B5E9E3771F7CF
:107CC000185F0F5FE394F7E0EF1609F084CFFF2011
:107CD00029F48091F7058F5F8093F7050F900F903F
:107CE000CF91DF911F910F91FF90EF90DF90CF9098
:107CF000BF909F908F907F906F9008958F929F92EA
:107D0000AF92BF92DF92EF92FF920F931F93CF93A8
:107D1000DF93F82E80E060E04DE659E021E00E941C
:107D2000924A4091B70A50E04F5F5F4F60E021E018
:107D30000E94B34BD090DD0A10E08091B70A8830E2
:107D400018F011E059E001C055E08DED9AE06F2D7B
:107D500040E020E030E000E0E52E0E94BB31809161
:107D6000B70A112369F090E00897EC01B3E0CC0F5B
:107D7000DD1FBA95E1F7C80FD91FCC52DB4F06C003
:107D800095E0899FE0011124C455DB4F00E1882470
:107D90009924AD2CBB24A7FCB094FE01E80DF91D7D
:107DA0004081552747FD509520E0A814B90409F4F7
:107DB00021E088E1602F0E94B34B0894811C911C44
:107DC000085F083351F7112319F485E090E01CC0D7
:107DD00000E1A5E08A2E912CFE01E80DF91D4081FD
:107DE000552747FD509520E0A814B90409F421E077
:107DF00080E3602F0E94B34B0894811C911C085FA4
:107E0000003351F789E090E020E0A816B90609F4A4
:107E100021E08CE068E346E659E00E94924A112393
:107E200019F485E090E002C089E090E0A816B90658
:107E3000ACF46D2D772767FD70956C0F7D1F8F2D2E
:107E40004CE95FEF24E630E002E00E94F00800E039
:107E50001CEFC0E0D0E0F0E2DF2E47C08F2D6CEDCC
:107E60007AE04CEF5FEF24E030E000E00E94F008A1
:107E7000882369F31123D9F020E73EEF8091DC0AD3
:107E8000992787FD9095AC01249FC001259F900DF7
:107E9000349F900D112460E170E00E944254699378
:107EA0002C593F4F51E0243F350741F71AC028E3D2
:107EB0003FEF8091DC0A992787FD9095AC01249FC4
:107EC000C001259F900D349F900D112468E070E053
:107ED0000E94425469932C593F4F51E02C32350790
:107EE00041F782E00E946243B2CFC8016091B70AB5
:107EF0000E94A20F9E014EE3240FF22EBC01E5E08A
:107F000076956795EA95E1F75D2D561B652F822FD3
:107F10000E94F44ACE0183709070009721F48F2D57
:107F200060E20E94F44A2196005E1F4FC034D105E2
:107F3000E1F68EE560E040E40E94ED4BDF91CF91E9
:107F40001F910F91FF90EF90DF90BF90AF909F90A7
:107F50008F9008952F923F924F925F926F927F92EF
:107F60008F929F92AF92BF92CF92DF92EF92FF9249
:107F70000F931F93DF93CF93CDB7DEB762970FB602
:107F8000F894DEBF0FBECDBF182F8091AD0A8823B5
:107F900019F44BEB58E002C045EC58E080E060E09B
:107FA00021E00E94924A9091AE0AC92EDD24C7FCBE
:107FB000D094F601EE0FFF1F960163E0220F331FEE
:107FC0006A95E1F7E20FF31FEA53FD4F8A5F60E025
:107FD000428D20E00E949D0D88EB9AE0612F40E0E9
:107FE00020E030E000E05CE0E52E0E94BB31209113
:107FF000B80A12161CF01092F70510C0822F9927AC
:1080000087FD90953091F705831B91098730910585
:108010000CF463C0822F86508093F705C601880F49
:10802000991FA3E0CC0CDD1CAA95E1F78C0D9D1DDA
:10803000F3EE6F2EF2E07F2E680E791EE4EE4E2EE8
:10804000E2E05E2E480E591E78EE272E72E0372EA3
:10805000280E391EAC014E515D4F5A834983FC01F5
:10806000EF51FD4FFC83EB8368E0F62E422F55273E
:1080700047FD50955E834D839C012A533D4FF90186
:108080007B96F887EF83A901445E5F4F5A87498743
:10809000F901B296FC87EB87BC0169517D4F5EE127
:1080A000852E912C820E931EA901435E5F4F5E8741
:1080B0004D87FC01E052FD4FF88BEF8745EEC42E53
:1080C00042E0D42EC80ED91E36EEA32E32E0B32ED7
:1080D000A80EB91E7A8B698B05C097FF9FCF20939E
:1080E000F7059CCF8091F70581509F2D9695969529
:1080F0009695890FEE24282F30E04D815E8142173E
:10810000530711F4EE24E394882321F18130E1F147
:10811000823009F46FC0833009F49AC0843009F4C6
:10812000C2C0853009F4F0C0863009F406C187303A
:1081300009F43AC1883009F465C1893009F485C170
:108140008A3009F4A0C18B3009F4BEC18C3009F02B
:10815000F5C1DBC18CE06F2D44EB58E020E00E94BC
:10816000924A8CE36F2DEF81F88540812E2D0E947D
:10817000AB0DEE2009F4E2C1812F6B817C8141E0DF
:1081800050E021E230E032C08CE06F2D4DEA58E043
:1081900020E00E94924AE985FA85408147FD02C0AD
:1081A00086E001C08BE0552747FD50959A0157FFA7
:1081B00004C022273327241B350B243614F09AE001
:1081C00005C02A3014F490E001C095E0845C890F6A
:1081D0006F2D2E2D0E94B34BEE2009F4AFC1812FDD
:1081E00069817A8143E85FEF2DE730E002E00E9489
:1081F000F008A4C18CE06F2D46EA58E020E00E9410
:10820000924AEB85FC85408147FD02C086E001C0B3
:108210008BE0552747FD50959A0157FF04C0222750
:108220003327241B350B243614F09AE005C02A307E
:1082300014F490E001C095E0845C890F6F2D2E2D21
:108240000E94B34BEE2009F479C1812FB101CACF4E
:108250008CE06F2D41EA58E020E00E94924AE989C3
:10826000FA898081817090E0AC01440F551F480F5E
:10827000591F4656574F8CE36F2D23E00E2D0E9459
:108280005C4AEE2009F45AC1E989FA89608161707B
:10829000812F40E021E00E940A0A8170E989FA8971
:1082A00090819E7F2FC18CE06F2D43E958E020E044
:1082B0000E94924AF401408183E0489FA00111246A
:1082C000435B574F8CE36F2D23E00E2D0E945C4AD9
:1082D000EE2009F433C1812FB20140E050E026E1E5
:1082E00030E002E00E94F008F4018081873008F459
:1082F00025C1103609F022C187508093B70A8EE756
:108300009EE30E942E0C1AC18CE06F2D46E458E0CB
:1083100020E00E94924A86E36F2DED85FE85408124
:108320002E2D0E94D60DEE2009F408C1812FB30135
:1083300040EF5FEF20E130E059CF8CE06F2D4EE34E
:1083400058E020E00E94924AEF85F8898781807F7B
:1083500091F0E989FA89408142954F7021F04A30C5
:1083600010F085E001C080E08E5B6F2D50E02E2D77
:108370000E94B34B07C08CE36F2D4AE358E02E2DCB
:108380000E94924AEE2009F4D9C0E989FA896081F5
:1083900062956F70812F40E023E00E940A0A829567
:1083A000807FE989FA894EC08CE06F2D43E358E065
:1083B00020E00E94924AE989FA89408146954770F7
:1083C00050E003E0440F551F0A95E1F7465E574F12
:1083D0008CE36F2D28E00E2D0E945C4AEE2009F4FC
:1083E000ADC0E989FA89608166956770812F40E0A8
:1083F00022E00E940A0A8770880FE989FA89908131
:10840000917F80C08CE06F2D4FE058E020E00E940B
:10841000924AF601408142954F7080E66F2D50E000
:108420002E2D0E94B34BEE2009F488C0F601608126
:1084300062956F70812F40E02FE00E940A0A8295BA
:10844000807FF60190819F705DC08CE06F2D46E0CB
:1084500058E020E00E94924AF60140814F7080E689
:108460006F2D50E02E2D0E94B34BEE2009F466C014
:10847000F60160816F70812F40E02FE00E940A0AB0
:108480008F70F6013DC08CE06F2D4BEF57E020E080
:108490000E94924AF501408142954F7080E66F2D0F
:1084A00050E02E2D0E94B34BEE2009F447C0F50199
:1084B000608162956F70812F40E02FE00E940A0A70
:1084C0008295807FF501BECF8CE06F2D42EF57E0A3
:1084D00020E00E94924AF50140814F7080E66F2DA6
:1084E00050E02E2D0E94B34BEE2041F1F50160814A
:1084F0006F70812F40E02FE00E940A0A8F70F50113
:108500009081907F982B908319C08CE06F2D40EE66
:1085100057E02E2D0E94924AEE2081F0103871F41F
:1085200080E80E94F74D8091AE0A0E9474258091E8
:108530003F0580933D0580E00E94680CF8E0FF0E47
:1085400020E4F21609F0CECD62960FB6F894DEBFA5
:108550000FBECDBFCF91DF911F910F91FF90EF9094
:10856000DF90CF90BF90AF909F908F907F906F9053
:108570005F904F903F902F900895CF92DF92EF92AF
:10858000FF920F931F93CF93DF93182F80E060E04B
:1085900040E259E021E00E94924A80EC9AE0612F8B
:1085A00048E026E833E008E0F7E0EF2E0E94BB3118
:1085B0002091C00AF22EFA941F141CF01092F705B5
:1085C00013C08F2D992787FD90953091F705831B58
:1085D00091098730910524F027502093F70504C0B6
:1085E00097FF02C0F092F705103859F01F3B11F4C5
:1085F0001092F70518E0EE24CF2CDD24C7FCD094B0
:1086000014C080E80E94F74D89E18093F90586E067
:10861000F81619F40E94BA4E03C08F2D0E94204F05
:1086200080913F0580933D05E5CF8091F7058E0D44
:10863000863071F1C82FD0E0CC16DD0611F024E0B1
:1086400001C025E0AE014F5F5F4F82E1612F02E084
:108650000E94124B8091F905882329F4CC16DD067F
:1086600011F421E101C020E1AE01E4E0440F551F07
:10867000EA95E1F74C1B5D0B4E575E4F88E1612F89
:108680000E94924AE394185F87E0E81671F611C0E1
:108690008091F905882311F020E005C020E086E0F4
:1086A000F81609F421E086E0612F4DE059E00E94C0
:1086B000924ADF91CF911F910F91FF90EF90DF9041
:1086C000CF900895882369F09091F30A982B9093A6
:1086D000F30A8091E00F9091E10F9093F50A809357
:1086E000F40A0895EF920F931F932091F30A222327
:1086F00009F466C0882309F05DC08091E00F909175
:10870000E10F4091F40A5091F50A841B950B8436D1
:10871000910508F455C04EC081EE9AE061E141E058
:108720002AE732E00CE410E074E1E72E0E94C04733
:108730008C34910511F480E020C08091E70A8230EA
:1087400021F48091F30A816023C084E899E02FC06E
:1087500081FF36C081EE9AE061E142E026EC32E032
:108760000BE612E054E1E52E0E94C04722E08B3672
:10877000920739F48091A7028F5F61E10E949746CA
:108780001FC08091E70A823081F48091F30A8260F1
:108790008093F30A8091E00F9091E10F845690400E
:1087A0009093F50A8093F40A0BC084E799E00E9445
:1087B000050C06C01092F30A822F20FFC9CFACCF60
:1087C0001F910F91EF9008950F931F93DF93CF9315
:1087D000CDB7DEB760970FB6F894DEBF0FBECDBF42
:1087E000682F6F5F062F0AC0102F1F5F812F688BC5
:1087F0000E9459456889882339F0012F0031A0F380
:10880000003111F480E025C081EE9AE00E947345AA
:10881000602F6F5F8AEE9AE042E028EC0E948E455E
:108820008E010F5F1F4F06C08AEE9AE0B8010E94CA
:108830003B47A89581EE9AE0B8014FE050E00E94D6
:10884000EF45482F882381F78AEE9AE00E94F94687
:1088500081E060960FB6F894DEBF0FBECDBFCF911A
:10886000DF911F910F91089581EE9AE060E00E94E0
:10887000734581EE9AE06AE772E04CE450E00E94B2
:108880004E488C34D1F480917A028330B1F4EBE716
:10889000F2E020E030E081919191280F391F82E0D1
:1088A000E339F807C1F780E04091A5025091A60294
:1088B0004217530719F481E0089580E00895AAE76C
:1088C000B2E08CE4FD0111928A95E9F783E0809390
:1088D0007A021092A70289E18093A8028AE5809328
:1088E000A90281E08093BE021196FD0120E032E0F2
:1088F00080E891E03183208397878687958F848FE6
:10890000329642E0E938F407A9F780E090E02D9133
:108910003D91820F931FE2E0A339BE07C1F7909308
:10892000A6028093A50208950F931F93CF93DF9320
:10893000EB01042F803180F5682F6F5F81EE9AE0A4
:108940000E94734510E0CE0160E270E0A8010E9431
:10895000B45481EE9AE0BE014AE050E00E944E48D5
:108960008A309105C9F481EE9AE00E9465459C0128
:10897000C00FD11F0EC0C9016AE070E00E942E54E2
:10898000805D8A93C9016AE070E00E942E54262F10
:10899000372F2115310579F7DF91CF911F910F9175
:1089A00008951F93182F86EC92E02BE632E0FC012D
:1089B000A901119241505040E1F763EB79E00E9428
:1089C0009B54212F30E02F5F3F4FC9016AE070E0D8
:1089D0000E944254605D6093CB02C9016AE070E07E
:1089E0000E944254805D8093CC0286E08093D00246
:1089F00080E00E94204F1F9108951F93182F80310F
:108A0000A8F4682F6F5F81EE9AE00E94734581EEB3
:108A10009AE066EC72E04BE652E00E944E4822E09B
:108A20008B36920719F0812F0E94D1441F9108952F
:108A3000EF920F931F930E946246882341F00E9499
:108A4000FA4887FD04C00E943444882351F583EA24
:108A500099E00E94050C0E94D3480E945F4481EE79
:108A60009AE060E041E02AE732E00CE410E0F8EC44
:108A7000EF2E0E94C0478C34910521F084E999E0E3
:108A80000E94050C80E00E94D14481EE9AE061E0F2
:108A900042E026EC32E00BE612E0E8ECEE2E0E941B
:108AA000C0478091A7020E94FD441F910F91EF9053
:108AB000089590E0FC01EE0FFF1FE80FF91FEA5048
:108AC000F54F8481811181E00895FC01808190E05F
:108AD000FC01EE0FFF1FE80FF91FE550F54F9181E4
:108AE00080819F700895FC0160831282118270E082
:108AF00026EF3AE0CB01880F991F860F971FD90107
:108B0000A80FB91F14964C911497438314821582B1
:108B10001682FD01868182958F700895CF93DF9331
:108B2000FC0160831282118270E0A6EFBAE0CB01F3
:108B3000880F991F860F971FED01C80FD91F3C8121
:108B40003383148215821682ED012696C80FD91F31
:108B50004295407F38813F70342B38831596A80F9B
:108B6000B91F1C9211968C911197807F11968C934E
:108B700011978091E00F9091E10F820F911D9087E6
:108B80008783DF91CF910895DF93CF930F92CDB775
:108B9000DEB7682F70E0E4E0660F771FEA95E1F733
:108BA000CE01019641E050E00E94BB5489810F90B4
:108BB000CF91DF910895EF92FF92CF93DF93809151
:108BC000F80AC0E0D0E003C02F960E94C445882375
:108BD000D9F7CE01DF91CF91FF90EF9008958F925A
:108BE0009F92AF92BF92CF92DF92EF92FF920F933C
:108BF0001F93DF93CF930F92CDB7DEB78C015B014C
:108C0000FC01808190E0FC01EE0FFF1FE80FF91FCF
:108C1000E550F54F80812181922F9F70F8012181CD
:108C20003281821B930BC42ED52E8C159D0508F422
:108C30006C0176014E010894811C911C27C0F8013B
:108C40006381662331F184818F5F848370E0F4E077
:108C5000660F771FFA95E1F7680F711DC40141E0B7
:108C600050E00E94BB548981F5018083F801848122
:108C70008F3030F0148283810E94C445F8018383D1
:108C80000894A11CB11C0894E108F108E114F10456
:108C9000B1F6F801818192818C0D9D1D8E199F097D
:108CA000928381838C2D8E190F90CF91DF911F912C
:108CB0000F91FF90EF90DF90CF90BF90AF909F907B
:108CC0008F90089586EF9AE060E070E040E450E015
:108CD0000E94BB548091F60A843011F080E0089520
:108CE00080E09091F70A903409F481E00895DF93D1
:108CF000CF930F92CDB7DEB76983682F70E0B4E0F1
:108D0000660F771FBA95E1F7CE01019641E050E07A
:108D10000E94DC4C0F90CF91DF91089586EF9AE08E
:108D200060E070E040E450E00E94DC4C0895DF9386
:108D3000CF9300D00F92CDB7DEB790E0FC01EE0FDD
:108D4000FF1FE80FF91FDE011196E650F54F23E0F3
:108D500001900D922150E1F770E0DC01AA0FBB1FDA
:108D6000A80FB91FFB01EE0FFF1FE60FF71FA6505C
:108D7000B54FE650F54F83E001900D928150E1F739
:108D8000FB01EE0FFF1FE60FF71FE650F54FDE0168
:108D9000119683E00D9001928150E1F70E948E467A
:108DA0000F900F900F90CF91DF91089588EF9AE088
:108DB00062E070E041E050E00E94DC4C08950F93C7
:108DC0001F93182F082F04C0802F0E94C445082F1E
:108DD000802F0E94C4458823B9F7802F6091F80A3C
:108DE0000E9477461093F80A0E94D6461F910F9171
:108DF00008951F93CF93DF93EC01888190E0FC01ED
:108E0000EE0FFF1FE80FF91FE550F54F89818083B2
:108E10009A819F708181807F892B81838B818823B8
:108E200089F00E94C445182F882361F08B8160E08F
:108E30000E9477460E948E46112331F0812F0E94B6
:108E4000DF4602C010E0F6CFDF91CF911F91089569
:108E50001F931091F80A112359F0812F0E94C445E5
:108E60008093F80A0E94D646812F60E00E947746E0
:108E7000812F1F910895AF92BF92CF92DF92EF9210
:108E8000FF920F931F93CF93DF93EC016B01F42EAE
:108E90008B81882389F489819A81009769F40881FC
:108EA00010E00E9428478B83F801EE0FFF1FE00FB0
:108EB000F11FEA50F54F84831F2D6FE0E62E46C068
:108EC0002091E00F3091E10F8F819885821B930BE9
:108ED00097FF02C082E004C08B81882319F481E0EF
:108EE0008E8337C09C819F3080F01C820E94C445D5
:108EF000882339F40B810E942847682F802F0E9415
:108F000077468B810E94C4458B838B81882339F3FC
:108F10006C819E2D961B012F911708F4092FA02E0E
:108F2000BB2470E06F5F7F4F90E054E0880F991F83
:108F30005A95E1F7680F791FC601A5010E94DC4C24
:108F4000CA0CDB1C8C81800F8C83101B112309F051
:108F5000B7CF2F2D30E0211B310989819A81820FF3
:108F6000931F9A8389838F2D811BDF91CF911F914E
:108F70000F91FF90EF90DF90CF90BF90AF9008954A
:108F80004F925F926F927F928F929F92BF92CF92F9
:108F9000DF92EF92FF920F931F93DF93CF930F9285
:108FA000CDB7DEB76C0129012E2D0E948E451982A6
:108FB0004201EE24FF2481E03E010894611C711CF3
:108FC000F4019081992351F4882319F0BB24B394C0
:108FD0000AC0F4019181992329F41AC0882311F061
:108FE000BB2409C0BB2499819F3718F4E016F10611
:108FF00059F5882379F08981882331F18068898344
:10900000C601B30141E00E943B478130E1F02BC033
:10901000BB24B39489818823B9F0C601B30141E030
:109020000E943B478130F9F44981B701641B710903
:10903000640D751DC6010E943B479981891719F07F
:10904000981B998310C019828B2D99819F5F9983FA
:109050000894E11CF11C0894811C911C0E151F053D
:1090600008F0AECF06C009810F77C701801B9109B8
:109070008C01C6010E94F946C8010F90CF91DF9183
:109080001F910F91FF90EF90DF90CF90BF909F9036
:109090008F907F906F905F904F9008958F929F92E6
:1090A000AF92BF92CF92DF92EF92FF920F931F93F6
:1090B000CF93DF938C015B016A01F5E08F2E912C39
:1090C000880E991EC0E0D0E03BC0F801858190E099
:1090D0008F779070009741F4C801B40141E050E0EF
:1090E0000E94EF45813079F5F8018581EFE7FE2E8A
:1090F000F8224F2D50E096012C1B3D0B241735070D
:1091000010F4FC2CFC1AB5016C0F7D1F87FF08C002
:10911000CB0160E070E04F2D50E00E94B4540AC0D3
:10912000C8014F2D50E00E94EF458F1519F0C80F70
:10913000D11D09C0CF0DD11DF80185818F198583FF
:10914000CC15DD0510F2CE01DF91CF911F910F916B
:10915000FF90EF90DF90CF90BF90AF909F908F9057
:109160000895DF93CF930F92CDB7DEB790E09C01C7
:10917000220F331F280F391FF901EA50F54F848160
:109180002650354F93E0D9011D929A95E9F78983CE
:109190000E948E468981882311F00E94DF460F903D
:1091A000CF91DF9108951F9380E4E6EFFAE0DF01AD
:1091B000982F1D929A95E9F794E09093F60A809380
:1091C000F70A1092F80A80E18093F90A84E0182FD8
:1091D0001F5F612F0E947746812F1038C1F78FE7FC
:1091E00060E00E94774684E08093F80A0E948E46F1
:1091F0001F910895CF92DF92EF92FF920F931F93EA
:10920000CF93DF9380E8E6E3FBE0DF011D928A95D0
:10921000E9F70AEF1AE0C0E0D0E08C2FC43139F44E
:10922000F090F80A98EFC92E9AE0D92E0BC06E0183
:10923000CC0CDD1CCC0EDD1E2AEF3AE0C20ED31E94
:10924000D801FC9090E0E82EE3941DC08F2D84504F
:109250008C3738F4EF2DF0E0EA5CF44F80818823FE
:1092600061F0992329F0892F60E00E9477460DC0B4
:10927000F60110820E948E4608C0E0828F2D0E9467
:10928000C4459F2DF82EFF2009F721960D5F1F4F33
:10929000C531D10511F614E0E12FF0E0EA5CF44F9E
:1092A0008081882349F4812F6091F80A0E947746D3
:1092B0001093F80A0E94D6461F5F103869F780E0C5
:1092C000DF91CF911F910F91FF90EF90DF90CF90A2
:1092D0000895EF92FF920F931F93CF93DF93EA01CC
:1092E0002196FA014491DE011196FE01E490FF24DB
:1092F000E7E0F0E0EE0EFF1E93E0F594E7949A9518
:10930000E1F7FD01949100FF02C051E010C001FDA2
:1093100002C050E00CC05091E20FC52FD0E016E023
:10932000D695C7951A95E1F7FE01E1705E2F11966B
:10933000929F90011124A20FB31F669566956695C2
:1093400070E09B013695322F22273795279590E0C4
:10935000280F391F6E0D7F1D7695762F662777951E
:109360006795680F791FC42FD0E01AC086EBE82EEE
:109370008BE0F82EE20EF31E80E090E00BC08D0132
:10938000080F191FF801049151110095F70101937D
:109390007F010196841798F3AC0FBD1F20583F4FF3
:1093A0002617370719F7DF91CF911F910F91FF9083
:1093B000EF9008950F931F93CF93DF936695669573
:1093C0006695062F10E01695102F00271795079524
:1093D000080F111D0A54144F85E04802A001112402
:1093E0004F5D564F20FF02C081E00DC021FD02C03D
:1093F00080E009C08091E20F90E036E09695879575
:109400003A95E1F7817027FF31C095E0992311F477
:1094100020E005C09A014F5F5F4FF901249181114F
:109420002095B8016F577F4FFFE0663B7F07D8F468
:1094300030E0E901CF70D070C152DE4FA881F80151
:10944000A183A083D90124E0B595A7952A95E1F7DA
:10945000A152BE4F2C91FB012083D801A058BF4FD1
:109460002C930E5F1F4F915088F61DC020E030E016
:10947000BA01620F731FFB019491FFE0063B1F07C7
:1094800028F481119095F80191938F012F5F3F4F40
:109490002530310569F7FFE0063B1F0720F48111F5
:1094A0008FEFF8018083DF91CF911F910F91089585
:1094B00020E00E94DA490895CF92DF92EF92FF9266
:1094C0000F931F93CF93DF93182FF62EE22EC42E07
:1094D000E6016E01D52EE601C02EDD2430E1C32267
:1094E000DD240FC0C114D10411F0488102C0FE0177
:1094F0004491812F6F2D202F0E94DA491A5FEA9440
:109500002196EE2079F7DF91CF911F910F91FF9077
:10951000EF90DF90CF9008950F9300E00E945C4A97
:109520000F910895DF92EF92FF920F931F93CF93C5
:10953000DF93182F062FD22EE42EE7017E01F52EA1
:10954000E701ED2CFF2430E1E322FF2401C0219646
:10955000E114F10411F0488102C0FE01449144235A
:1095600051F0812F602F2D2D0E94DA491A5FD7FE0E
:10957000EECF1A5FECCF812FDF91CF911F910F912A
:10958000FF90EF90DF90089520E00E94924A0895A6
:10959000EF92FF920F931F93DF93CF930F92CDB76C
:1095A000DEB7182F062F7A01982F9C5E95504E2D0E
:1095B0004F704A3014F0495C01C0405D892F602F24
:1095C00099830E94584A9981911731F064E0F6948A
:1095D000E7946A95E1F7EACF0F90CF91DF911F9161
:1095E0000F91FF90EF900895E62FE695E695E695AA
:1095F000F0E0F695FE2FEE27F795E795E80FF11DC1
:10960000EA54F44F8FE0E63BF80758F4677021E026
:1096100030E002C0220F331F6A95E2F78081822773
:10962000808308952F923F925F926F927F928F92E4
:109630009F92AF92BF92CF92DF92EF92FF920F93E1
:109640001F93DF93CF930F92CDB7DEB7F62E1A019B
:10965000122FC02E27FF03C09AE0E92E02C005E0BA
:10966000E02EA12EBB24992437FE06C099249394A2
:1096700030942194310833949501B5E035952795C0
:10968000BA95E1F7322F3370082F0650DD24A7E09A
:109690008A2E8F0CF6E05F2E5F0CE4E06E2E712CAC
:1096A0006A207B203BC03323D9F03D15C9F401501B
:1096B000C1016AE070E00E944254482F405D802F53
:1096C0006F2D212F0E94DA49802F8B5F682D0E9419
:1096D000F44A802F8A5F652D0E94F44A30E00EC064
:1096E000C1016AE070E00E944254482F405D802F23
:1096F0006F2D212F39830E94DA493981C1016AE037
:1097000070E00E9442541B016114710429F4211479
:10971000310411F4332321F00E19D394DC1418F220
:10972000992029F0802F8E196F2D4DE206C0A3FEDF
:1097300007C0802F8E196F2D4BE2212F0E94DA492E
:109740000F90CF91DF911F910F91FF90EF90DF90DD
:10975000CF90BF90AF909F908F907F906F905F90D1
:109760003F902F9008950F9305E00E94124B0F91A8
:10977000089520E00E94B34B089547FF02C0840F74
:109780004195E62FE695E695E695F0E0F695FE2FF5
:10979000EE27F795E795E80FF11DEA54F44F67704F
:1097A00081E090E0382F01C0330F6A95EAF7632F0C
:1097B0000DC0822F90E09C013595279580FF04C055
:1097C000808186278083206841503196442389F721
:1097D00008952FEF0E94BD4B08950F931F93CF93D1
:1097E000DF93082F10E0E62FE695E695E695F0E08A
:1097F000F695FE2FEE27F795E795E00FF11FEA5457
:10980000F44FC62FD0E0242F332727FD30952C0F9F
:109810003D1FC90168E070E00E9442547695762FA2
:10982000662777956795600F711F6A54744FC770EC
:10983000D07081E090E00C2E02C0880F991F0A942E
:10984000E2F7982F91958081892704C0E058FF4F57
:10985000808180958083E617F707C0F3C90168E02F
:1098600070E00E94425421E030E002C0220F331F1A
:109870008A95E2F72195808182278083DF91CF91BD
:109880001F910F910895A998AB98AC988BBBAD9A96
:10989000AD98AB9AA99A0895A998AB9AAC988BBB4E
:1098A000AD9AAD98AB9AA99A0895BC0120E030E03A
:1098B00045E005C0942F9A95F1F72F5F3F4F26178B
:1098C0003707C4F30895AA9885E0982F9A95F1F781
:1098D0008A95F1F7AA9A80E090E035E0232F2A9547
:1098E000F1F7019625E08C3D9207C1F782EE0E94C8
:1098F000434C8EEA0E94434C81EA0E94434C86EA24
:109900000E94434C84EA0E94434C82EA0E94434CEA
:1099100080EC0E94434C8FE20E94434C85E20E94FF
:10992000434C81E80E94434C82E20E94434C8FEA00
:109930000E94434C82E28093A80208951F93182F3F
:1099400081E80E94434C812F0E94434C1F9108954F
:10995000EF92FF920F931F93CF93DF93C6EBDBE061
:1099600010E07E0184E00E94434C80E10E94434C61
:10997000812F806B0E94434C00E0F70181917F01B1
:109980000E944C4C0F5F0038C1F71F5FC058DF4F7B
:10999000183039F7DF91CF911F910F91FF90EF9021
:1099A000089580E094E0E6EBFBE0DF019C011D926E
:1099B00021503040E1F70895E82FF92F862F972F97
:1099C00013C02081E199FECF9FBB8EBBE09A3DB3CF
:1099D000231731F02DBB2FB7F894E29AE19A2FBFED
:1099E00031960196415050404115510551F7089567
:1099F0008093E30F08958091E30F1092E30F089591
:109A0000FC018081982F990F9E70807F892B808325
:109A1000662321F09160807F892B808381818F5F15
:109A200081839281992391F020812F7079F493366C
:109A300059F0242F20622093E30F903111F48031EC
:109A400018F080818F7C808311821282828188232A
:109A500081F08130E1F1823091F1843081F1883000
:109A600071F1803129F1813689F0823609F042C0E6
:109A70003BC08081982F9F709F30E1F591E69283E3
:109A80009181913198F08F7C808310C04066409323
:109A9000E30F9081892F82958F708F5F83708295FD
:109AA000807F9F7C982B908380E182831182089530
:109AB0009181983121F4942F90689093E30F9181D4
:109AC000903328F090E0959587958283118282816A
:109AD00090E00197218130E082239323009751F495
:109AE00040644093E30F08958181803418F088E04A
:109AF0008283118208959C018E3091057CF480E070
:109B0000F901EE0FFF1FE20FF31FEA54F04F9081AF
:109B10009F709F3009F05BC081E008958E30910501
:109B200009F443C08F30910511F18031910599F00E
:109B300081319105F9F08231910511F1833191055F
:109B400029F18431910571F08531910531F186312A
:109B50009105E1F532C081B190E096958795969593
:109B6000879532C083B3881F8827881F0895809106
:109B700063002AC0809163008695869586950BC008
:109B80008091630083FF22C081B110C081B18295B2
:109B9000869586958370809517C081B190E054E0DA
:109BA000969587955A95E1F70FC083B390E046E00C
:109BB000969587954A95E1F707C081B190E035E029
:109BC000969587953A95E1F78170089580E008951C
:109BD0008F708E3058F490E0FC01EE0FFF1FE80FFD
:109BE000F91FEA54F04F82E68283118208958F7044
:109BF0008E3068F490E0FC01EE0FFF1FE80FF91FB4
:109C0000EA54F04F83E6828380818F7C80830895BD
:109C10008F708E3010F080E0089590E0FC01EE0F20
:109C2000FF1FE80FF91FEA54F04F8081829583707F
:109C300008950F931F93CF93DF938091E00F90913E
:109C4000E10F01969093E10F8093E00F8091E20F76
:109C50008F5F8093E20F06B3009540E050E010E084
:109C6000EA012196CA01880F991F840F951FB80138
:109C70000C2E02C0759567950A94E2F761707070BA
:109C80008A54904F50E00E94004DAE01C630D1057D
:109C900039F710B31095C0E0D0E0FE01EF55F44F56
:109CA0002491CE01880F991F8C0F9D1F8853904FD0
:109CB00060E0212309F061E09E012A5F422F50E01D
:109CC0000E94004D2196C830D10539F7DF91CF9120
:109CD0001F910F910895FB01282F30E0883018F56F
:109CE000C901880F991F880F991F820F931F8A53EC
:109CF0009D4FDC01AA51BE4F20812C93DC01A9515C
:109D0000BE4F21812C93DC01A851BE4F22812C93A0
:109D1000DC01A751BE4F23812C9386519E4F248195
:109D2000FC0120830895DB0128503040F90193E0C5
:109D3000EE0FFF1F9A95E1F7E20FF31FEC52FB4F76
:109D400099E0899FC00111248B569B4F2D9121933F
:109D5000E817F907D9F70895ECEAF4E088E2DF01A3
:109D60001D928A95E9F7B89688E4DF011D928A95DD
:109D7000E9F7089580E491E0E0EEF2E0DF019C0174
:109D80001D9221503040E1F70895EF92FF920F931A
:109D90001F93CF93DF93F82EE0EEF2E080E090E0A7
:109DA000582F9C014081F41638F0442329F0019685
:109DB0003A9681329105A1F7503219F4C0EED2E003
:109DC00037C08901000F111FC901A3E0880F991F37
:109DD000AA95E1F7080F191FE801C052DD4FA9014C
:109DE0004F5F5F4FCA01880F991FE3E0440F551F73
:109DF000EA95E1F7840F951F20953095205E3F4F3F
:109E0000A901440F551F63E0220F331F6A95E1F744
:109E1000420F531F80529D4FBE010E94A2548AE000
:109E2000FE0111928A95E9F7F801EA53FD4FF28E8F
:109E3000CE01DF91CF911F910F91FF90EF90089588
:109E40006F927F928F929F92AF92BF92CF92DF924A
:109E5000EF92FF920F931F93DF93CF93CDB7DEB7AF
:109E600069970FB6F894DEBF0FBECDBF182F8823B9
:109E700081F0813009F47AC0823009F48EC08330D9
:109E800009F4FFC0843009F470C1853009F02BC497
:109E900032C2E091C302F0E0EE0FFF1FEE0FFF1F92
:109EA000E151FE4F81810E94C54EDC01E091BE026E
:109EB000F0E0EE0FFF1FEE0FFF1FE15BFD4F808113
:109EC00011968C93119714E612961C93E091C3029D
:109ED000F0E0EE0FFF1FEE0FFF1FEF50FE4F8081EF
:109EE0000E94C54EDC01E091BE02F0E0EE0FFF1FC4
:109EF000EE0FFF1FE15BFD4F818111968C9311974F
:109F000012961C93E091C302F0E0EE0FFF1FEE0FDC
:109F1000FF1FE151FE4F83810E94C54EDC01E0919D
:109F2000BE02F0E0EE0FFF1FEE0FFF1FEF5AFD4FD6
:109F3000808111968C93119712961C93E091C30225
:109F4000F0E0EE0FFF1FEE0FFF1FED50FE4F808180
:109F50000E94C54EDC01E091BE02F0E0EE0FFF1F53
:109F6000EE0FFF1FE15BFD4F838184C0E091C302D0
:109F7000F0E0EE0FFF1FEE0FFF1FE151FE4F838158
:109F80000E94C54EFC0188E081838CE982831383A3
:109F90008781817F84608783A6C3E091C302F0E05C
:109FA000EE0FFF1FEE0FFF1FE151FE4F81810E9458
:109FB000C54EDC01E091BE02F0E0EE0FFF1FEE0F98
:109FC000FF1FE15BFD4F808111968C93119714E682
:109FD00012961C93E091C302F0E0EE0FFF1FEE0F0C
:109FE000FF1FE151FE4F81810E94C54EDC01E091CF
:109FF000BE02F0E0EE0FFF1FEE0FFF1FE15BFD4F13
:10A00000818111968C9311978CE912968C93E09133
:10A01000C302F0E0EE0FFF1FEE0FFF1FEF50FE4FE9
:10A0200080810E94C54EDC01E091BE02F0E0EE0F9F
:10A03000FF1FEE0FFF1FE15BFD4F808111968C9398
:10A04000119712961C93E091C302F0E0EE0FFF1FF0
:10A05000EE0FFF1FEF50FE4F80810E94C54EDC01C6
:10A06000E091BE02F0E0EE0FFF1FEE0FFF1FE15B7D
:10A07000FD4F818111968C93119712961C93129724
:10A0800032C3E091C302F0E0EE0FFF1FEE0FFF1F9F
:10A09000EF50FE4F80810E94C54EDC01E091BE0270
:10A0A000F0E0EE0FFF1FEE0FFF1FE15BFD4F818120
:10A0B00011968C93119714E612961C93E091C302AB
:10A0C000F0E0EE0FFF1FEE0FFF1FEF50FE4F8081FD
:10A0D0000E94C54EDC01E091BE02F0E0EE0FFF1FD2
:10A0E000EE0FFF1FE15BFD4F838111968C9311975B
:10A0F00012961C93E091C302F0E0EE0FFF1FEE0FEB
:10A10000FF1FED50FE4F80810E94C54EDC01E091A3
:10A11000BE02F0E0EE0FFF1FEE0FFF1FE15BFD4FF1
:10A12000818111968C93119712961C93E091C30232
:10A13000F0E0EE0FFF1FEE0FFF1FED50FE4F80818E
:10A140000E94C54EDC01E091BE02F0E0EE0FFF1F61
:10A15000EE0FFF1FE15BFD4F838111968C931197EA
:10A160008CE912968C931297BEC2E091C302F0E084
:10A17000EE0FFF1FEE0FFF1FEF50FE4F80810E947A
:10A18000C54EDC01E091BE02F0E0EE0FFF1FEE0FC6
:10A19000FF1FE15BFD4F818111968C93119788E43D
:10A1A00012968C93E091C302F0E0EE0FFF1FEE0FCA
:10A1B000FF1FEF50FE4F80810E94C54EDC01E091F1
:10A1C000BE02F0E0EE0FFF1FEE0FFF1FEF5AFD4F34
:10A1D000808111968C93119717E312961C93E0914E
:10A1E000C302F0E0EE0FFF1FEE0FFF1FED50FE4F1A
:10A1F00080810E94C54EDC01E091BE02F0E0EE0FCE
:10A20000FF1FEE0FFF1FE15BFD4F818111968C93C5
:10A2100011970CED12960C93E091C302F0E0EE0F53
:10A22000FF1FEE0FFF1FED50FE4F80810E94C54EB5
:10A23000DC01E091BE02F0E0EE0FFF1FEE0FFF1F0A
:10A24000E15BFD4F838111968C9311978EE31296FB
:10A250008C93E091C302F0E0EE0FFF1FEE0FFF1FA3
:10A26000ED50FE4F80810E94C54EDC01E091BE02A0
:10A27000F0E0EE0FFF1FEE0FFF1FEF5AFD4F808142
:10A2800011968C93119712961C9386E00E94C54EEE
:10A29000DC01E091BE02F0E0EE0FFF1FEE0FFF1FAA
:10A2A000E15BFD4F818111968C93119712960C936F
:10A2B00086E00E94C54EDC01E091BE02F0E0EE0FA8
:10A2C000FF1FEE0FFF1FE15BFD4F838111968C9303
:10A2D000119782EC12968C9386E00E94C54EDC01A9
:10A2E000E091BE02F0E0EE0FFF1FEE0FFF1FEF5AEE
:10A2F000FD4F8081BFCE0E94BA4E0E94AC4EE091CD
:10A30000C302F0E0EE0FFF1FEE0FFF1FED50FE4FF8
:10A3100080810E94C54EFC010AE1C02EC182B2E3D9
:10A320007B2E7282E091C302F0E0EE0FFF1FEE0F72
:10A33000FF1FED50FE4F80810E94C54EFC017BE166
:10A34000872E81826CE9E62EE282E091C302F0E082
:10A35000EE0FFF1FEE0FFF1FED50FE4F80810E949A
:10A36000C54EFC014CE1D42ED18204E602838781E4
:10A3700081608783E091C302F0E0EE0FFF1FEE0FD4
:10A38000FF1FEF50FE4F80810E94C54EFC01C1822D
:10A39000E282E091C302F0E0EE0FFF1FEE0FFF1F1D
:10A3A000EF50FE4F80810E94C54EFC01D182028396
:10A3B000878181608783E091C302F0E0EE0FFF1F89
:10A3C000EE0FFF1FE151FE4F83810E94C54EFC013D
:10A3D000A091BE02B0E0AA0FBB1FAA0FBB1FAF5ACD
:10A3E000BD4F8C918183028374E0972E938267E046
:10A3F000662E6482878181608783E091C302F0E0EA
:10A40000EE0FFF1FEE0FFF1FE151FE4F83810E94F1
:10A41000C54EFC01A091BE02B0E0AA0FBB1FAA0F5F
:10A42000BB1FAF5ABD4F8C9181830283138338E0E9
:10A43000F32EF482878181608783E091C302F0E08C
:10A44000EE0FFF1FEE0FFF1FE151FE4F83810E94B1
:10A45000C54EFC01A091BE02B0E0AA0FBB1FAA0F1F
:10A46000BB1FAF5ABD4F8C9181838EE6828386E0FD
:10A47000A82EA382F482878181608783E091C30242
:10A48000F0E0EE0FFF1FEE0FFF1FE151FE4F838143
:10A490000E94C54EFC01F18283E88283BB24B39401
:10A4A000B3828781817F85608783E091C302F0E07A
:10A4B000EE0FFF1FEE0FFF1FE151FE4F81810E9443
:10A4C000C54EDC01E091BE02F0E0EE0FFF1FEE0F83
:10A4D000FF1FE15BFD4F808111968C9311971296BF
:10A4E0000C9385E00E94C54EFC01F182728288EFD8
:10A4F000838387818160878385E00E94C54EFC014C
:10A50000F1826EEC762E7282F3828781816087837E
:10A5100085E00E94C54EFC01618288E282838781CA
:10A520008160878386E00E94C54EFC01C1827282F1
:10A5300086E00E94C54EFC018182E28286E00E9494
:10A54000C54EFC01D182E28287818160878389E0E8
:10A550000E94C54EDC01E091BE02F0E0EE0FFF1F4D
:10A56000EE0FFF1FE15BFD4F818111968C931197D8
:10A570008CE312968C938AE00E94C54EDC01E09138
:10A58000BE02F0E0EE0FFF1FEE0FFF1FE15BFD4F7D
:10A59000838111968C9311978CEC12968C938BE09F
:10A5A0000E94C54EFC01A091BE02B0E0AA0FBB1FE5
:10A5B000AA0FBB1FAF5ABD4F8C91818326E4F22EA8
:10A5C000F282938289E084838781816087838BE034
:10A5D0000E94C54EFC01A091BE02B0E0AA0FBB1FB5
:10A5E000AA0FBB1FAF5ABD4F8C918183F282138398
:10A5F0001AE014838781816087838BE00E94C54EB7
:10A60000FC01A091BE02B0E0AA0FBB1FAA0FBB1FA6
:10A61000AF5ABD4F8C918183F282A38214838781CC
:10A62000816087838BE00E94C54EFC01A091BE0231
:10A63000B0E0AA0FBB1FAA0FBB1FAF5ABD4F8C9132
:10A6400081830283B3828BE084838781807F8560EE
:10A650008783DE011196E3E7F2E085E001900D9239
:10A660008150E1F7DE011696EEE6F2E085E001901A
:10A670000D928150E1F7DE011B96E9E6F2E085E0FC
:10A6800001900D928150E1F7DE015096E4E6F2E090
:10A6900085E001900D928150E1F7DE015596EFE5DE
:10A6A000F2E085E001900D928150E1F7BE016F5F0D
:10A6B0007F4F0E946B4E81E0BE016A5F7F4F0E9418
:10A6C0006B4E82E0BE01655F7F4F0E946B4E83E060
:10A6D000BE01605F7F4F0E946B4E84E0BE016B5EE7
:10A6E0007F4F0E946B4E82E00E94624369960FB6D4
:10A6F000F894DEBF0FBECDBFCF91DF911F910F91B8
:10A70000FF90EF90DF90CF90BF90AF909F908F9091
:10A710007F906F9008951F920F920FB60F921124A1
:10A720002F938F939F93EF93FF938BB12AB19CB19B
:10A730008C7121F421FD0DC09E3F29F4109204106C
:10A740001092051012C09F3F81F481E080930410A5
:10A750000CC080910510803240F4E82FF0E0EC51FD
:10A76000F04F90838F5F80930510FF91EF919F9141
:10A770008F912F910F900FBE0F901F90189580EF23
:10A7800090E0909379028093780210981898109234
:10A79000900087E689B9599886E38093950084E014
:10A7A0008AB901C08CB15F99FDCF0895539808957F
:10A7B000539A0895549857980895549A579A08951B
:10A7C0005D9BFECF509890FD509A8CB908955D9B8B
:10A7D000FECF509A8CB9089505C05D9BFECF509A6C
:10A7E0002CB90196FC0120812223B9F708955D9BC5
:10A7F000FECF50988EEF8CB908955D9BFECF509898
:10A800008FEF8CB90895629FD001739FF001829FF2
:10A81000E00DF11D649FE00DF11D929FF00D839FEF
:10A82000F00D749FF00D659FF00D9927729FB00D8C
:10A83000E11DF91F639FB00DE11DF91FBD01CF019F
:10A8400011240895991B79E004C0991F961708F008
:10A85000961B881F7A95C9F780950895AA1BBB1B84
:10A8600051E107C0AA1FBB1FA617B70710F0A61B10
:10A87000B70B881F991F5A95A9F780959095BC0131
:10A88000CD01089597FB092E07260AD077FD04D045
:10A89000E5DF06D000201AF4709561957F4F08958A
:10A8A000F6F7909581959F4F0895A1E21A2EAA1B65
:10A8B000BB1BFD010DC0AA1FBB1FEE1FFF1FA21770
:10A8C000B307E407F50720F0A21BB30BE40BF50B6D
:10A8D000661F771F881F991F1A9469F760957095F6
:10A8E000809590959B01AC01BD01CF01089597FB28
:10A8F000092E05260ED057FD04D0D7DF0AD0001C44
:10A9000038F450954095309521953F4F4F4F5F4F0C
:10A910000895F6F790958095709561957F4F8F4FCC
:10A920009F4F0895FB01DC0102C005900D9241503C
:10A930005040D8F70895FB01DC0105900D920020EE
:10A94000E1F708956817790768F4FB01DC01E40F6B
:10A95000F51FA40FB51F02C002900E924150504047
:10A96000D8F708950C94CB54DC0101C06D9341508D
:10A970005040E0F70895DC01CB01FC01E199FECFE6
:10A9800006C0FFBBEEBBE09A31960DB20D9241506E
:10A990005040B8F70895FB01DC0102C001900D9210
:0CA9A00041505040D8F70895F894FFCFC4
:10A9AC0088064F062206CE07FF07010203040103A7
:10A9BC000204040203010403020100010100220449
:10A9CC007C5E01020304010204030103020401037F
:10A9DC000402010402030104030202010304020144
:10A9EC000403020301040203040102040103020430
:10A9FC000301030102040301040203020104030224
:10AA0C000401030401020304020104010203040112
:10AA1C000302040201030402030104030102040300
:10AA2C00020153696D706C6520342D4348000000A1
:10AA3C0000542D437574000000000000000000005D
:10AA4C00562D5461696C00000000000000000045A8
:10AA5C006C65766F6E5C44656C74610000006543D8
:10AA6C0043504D0000000000000000000048656CE1
:10AA7C00692053657475700000000000000201002D
:10AA8C00030C0F30333C3FC0C3CCCFF0F3FCFF01C1
:10AA9C000203040102040301030204010304020182
:10AAAC000402030104030202010304020104030271
:10AABC000301040203040102040103020403010361
:10AACC000102040301040203020104030204010352
:10AADC000401020304020104010203040103020441
:10AAEC000201030402030104030102040302010135
:10AAFC000203040103020404020301040302019C87
:10AB0C00000000649CC4003C64ECEC003C645A46BD
:0AAB1C0032465A9C1432465AF000EB
:00000001FF
